:100000000C9456260C94D32D0C94AC2D0C94492DA5
:100010000C94E62C0C94752C0C947E260C947E2665
:100020000C947E260C947E260C947E260C94FA2D3D
:100030000C947E260C947E260C947E260C947E26B0
:100040000C946A290C947E260C941D280C94F72796
:100050000C947E260C947E260C947E260C947E2690
:100060000C947E260C947E26752A782A7B2A7E2A7A
:10007000812A842A872A8A2A8D2A902A932A962AD4
:10008000992A9C2A9F2AA22AA52AA82AAB2AC92AE9
:10009000AE2AB12AB42AB72ABA2ABD2AC02AC32A4C
:1000A000C62AC92AC92ACC2ACF2AD22AD52AD82A8E
:1000B000DB2ADE2AE12AE42AE72AEA2AED2AF02AC4
:1000C000F32AF62AF92AFC2AFF2A022B052B082BF1
:1000D0000B2B1A2B1D2B202B232B262B292B2C2BC8
:1000E0002F2B322B352B382B3B2B3E2B412B442BEC
:1000F000472B4A2B4D2B502B532B562B592B5C2B1C
:100100005F2B622B652BF82BFB2BFE2B012C042C79
:10011000072C0A2C262C292C2C2C2F2C322C352C5D
:10012000382C3B2C3E2C412C442C472C4A2C4D2C5B
:10013000502C532C562C592C5C2C173529355E35F8
:10014000CB35DF35F1350236263646367436D936AC
:10015000593765370F3849388038B838C83840358E
:100160004335463549354C354F355235553558357B
:100170005B357D3580358335863589358C358F35D2
:100180009235953598359B359E35A135A435A735E3
:10019000AA35AD35B035B335B635B935BC35BF3513
:1001A000C235C535C8358437A737B237BD37C437F0
:1001B000D337D637E137EC37EF37FA370538083819
:1001C0006238653868386B386E387138743877380B
:1001D0007A387D3807634236B79BD8A71A396856F4
:1001E00018AEBAAB558C1D3CB7CC5763BD6DEDFD59
:1001F000753EF6177231BF000000803F0800000016
:10020000BE922449123EABAAAA2ABECDCCCC4C3E0B
:1002100000000080BEABAAAAAA3E00000000BF00FA
:100220000000803F0000000000084178D3BB4387F6
:10023000D1133D190E3CC3BD4282AD2B3E68EC820A
:1002400076BED98FE1A93E4C80EFFFBE01C4FF7F8F
:100250003F000000000009582A2500CB9F956C1430
:100260002189A978B35BECBAB523134697993ED69A
:10027000B92E79C95BD84741531FC7E19C855422E9
:10028000ECFADBDD239349B8E678FF3F0998DA22E0
:100290000137781A2085D1503A3311815D5B95D4AE
:1002A0004404769DD5A93AABF0A13EB7BAD5A92BA7
:1002B000EBCCA03EB7BDC35A3BC86967BDFBE8673E
:1002C000BFCA9DE97408E7CE777806893257D6F120
:1002D000F18F7DFE1FA5EFD6503B678FB93B2349B9
:1002E0007F3387310CE922497D56DF69AA396D5980
:1002F000DD825692DAE5749DA7A6D39A53379956B4
:10030000A66F4F599D7B892FDDC528AA154BA3D613
:10031000AE8C8AAD543BA7A93BB3545D33E6A65CD3
:10032000CB75CD5EC6DAA4CAB935AE67B84640B65D
:1003300028BBF1F6B7B94720B628BBFF0F0E383CF3
:100340002D005FB61960A89093362BE299B34ED971
:100350007D89852FBED5AD4F3F64ABA43EBAD3593E
:100360009A2E75D5396D6B0A2D3CECE5DD1FFEB07C
:10037000E7FF0308684E9D021C60C08C6912B0C084
:1003800028AB8C9CC02DBB38793115A3B6E416B7C9
:10039000DCF56E57DF545B85BED9E35CC6D66DB124
:1003A000A5BF995B3B5A3009AF2FEDEC31C45CBE61
:1003B000D633DDAD8887E2D2F2F4E0162AB2E363E9
:1003C0001FF9F0E7FF010CE82E94014DBA4A4003F3
:1003D000166869361CE9BAB8E539707284DB51A435
:1003E000A84EA3C977B1CAD652A871ED2A7B4BA6F5
:1003F000E037B75ADD488E94F164CE6D195591BC43
:100400006ED7AD1EF5AA777AC67022CDC7F989CF0F
:10041000FF0306B859340027D6386058D391552DBC
:10042000AA659D4FD1B8391767BFC5AE5A1DB57AB9
:1004300006F6A97D9DD26C55A52675C99BDFFC6E7D
:100440000E633A3470AF3EFF1FE6A81A355DD69AA8
:10045000354B8C4E6B1AD6A651B2B5EE589A134F47
:10046000B5356768263D4D979CBEC9752F6D7BBB22
:100470005BDFFA36A7EFBA25DA16DF69AC2305454C
:10048000F9ACB98FA39720739F54CE1E45C2A24EDC
:100490003ED3D53DB179240DD7484C6EE12CDEFF1B
:1004A0000F656989C57366DFE98C330E41C6EA5B67
:1004B000EF7AF5332550E5EA39D7C56E0814C1DD6A
:1004C000456403008000AE7033C073331A10408F50
:1004D0002B14F87F0CF85E4C01BF957BC00216B060
:1004E000C0C8BA364DB72737BBC529BA716DB7B585
:1004F000ABA8CEBDD4DEA6B25AB1346A1DA735373B
:10050000E55AAE6BEED2B6264C37F54DB99A343972
:10051000B7C6E11E81D8A2ECE6C77FFEFB7F04F8D8
:10052000AD4C0216B0800656355DA82A6DB9CD696E
:10053000BB2B55B52DB7DBFD9C0DD8328A7BBC0299
:1005400000030CB12E80DFD23520010E60E0FF01E8
:1005500008983193021CE080075AD61C6B782EBD98
:10056000E52D4FDDADABAA6DC92302564C930005B6
:1005700010908931FC3F01D8B6DD012FF43860D5E9
:10058000D1914D9784E64B4E36B21067CD19D92CD8
:100590000194F1786633EB79AF7B578736AF520819
:1005A0009E6BEA5AB77A94734547AC5A9CAFFF07E3
:1005B00004A8BE5C00DDA511A0FA72027497C60102
:1005C000099CA6AB300DCE7AEA6A4A3935FBAA8B74
:1005D0001BC676F7AB2E7919CAD5EFCA570814A1F6
:1005E000DC45640300C0FF030AE84ACD01DBB933F0
:1005F000C0A6540CA434D9F20A6CBBB3530E5DA64A
:10060000259B6F75CA6152DC7449A98AC4764DD79F
:10061000B176C055A665D826995C56ADB92523D5C7
:100620007C3296E99B207DCB3CFA55AE991A30FC82
:100630004B3CFF1F04C87E5C020AA8624303A7A8C4
:1006400062434B97DCF214C5A79B7AD39537C31E40
:10065000164A6636F35A896ED43055B532B731B57D
:10066000C1692CE9F7BC961239D4B5FDDA9B0FD1DC
:1006700090EEF5E4170245287711D9409E45DD2B11
:1006800033717ABA0B13952DF9F97FA96B21B92231
:10069000669FAEC7E1707B72BB5BDFEA56BB5C65F1
:1006A000CB66C53D67D7AB6D2E643093EEB1CD3DC3
:1006B00092B99ADAB28E40129A6AEB968F7898B312
:1006C0002AB4D348AA2F7DA77BFB0C73715CCE6E36
:1006D0005C526C73799A134B8945E96E4942A9576C
:1006E000FF3F0CE82ED4020698D2550316687D17FA
:1006F000E96EBC658C456DA6E996DDDEF6B6B75EA3
:1007000075D493A59C7B57B36E7D1219ADDC298DF2
:100710004F93B487D2B6FCDDAC2256027018CA18CB
:1007200026B590D4DE6B29DA2D25178D7988D4482B
:10073000795DF77475A194A9D1F2ED9EAA51A6D462
:100740009E7FED6FFE2BD1C73D89FAB70D57D3B40D
:10075000F53755372EE6B2D757FF0F69FB59DD51F4
:10076000D5D7B56F0A78C052010F50ACF6A8161550
:10077000F27BEA1947D064EBAD76B5EBD196246EE7
:10078000626D5B1F0AA7B9C5ABFD1A62F0F0E26C9F
:10079000731C73521D19946FCE7DED6BD982DC48AA
:1007A000C72E718BBBDFFF1FE628C4F8449AFBCD30
:1007B000AD8D2A4E4ABCB88CB98AA948ED7287D350
:1007C000743B1AA99D6FB3CA5E8CC37BF2CE5A5E8E
:1007D00035665A3AAE55EB9A5775A9296BEEB6D5E0
:1007E0004D37EFB55DC59584E5A6FC30E0970C0D5F
:1007F0005840031CA0C0FF036DFEDEC4C4E829609E
:10080000002E0F9C6C29712A4E779315772AAEC360
:10081000CE763C92A54478D16DCF473BB8BB07F666
:100820005B43916EA9F2654CC99897699FBAE5330D
:100830009CC19A8FCADE70079DEEC979E2EDFFFF79
:10084000076EEF4258B66BA77D6825CC59B4F611F8
:1008500082C86AF11A462E128D37A7EFC9C9A36E56
:100860009F76D422737FB4EA510B2D62E2A84743EE
:10087000D72E29AE4D92AA285C8BB96AEB2495E35A
:10088000801D933590BA590345B37519462796983C
:10089000C5651FCD88BC16D73D3D6310496EEDF888
:1008A000FAEFFF01ABAADEB462669FA27573D36E46
:1008B00072B25654CBBAB60192C726404B430CC80D
:1008C00029C501CFB81AE0A71407FC56EA0105981C
:1008D000605AEAD429B5B8EB685317B3966EA32FC4
:1008E00029545BF68DB5A9325EDB37B6A1DBB17456
:1008F000CB58BA4991F6CDE31A3A853A56B76B9878
:1009000062EAF8DCBE9E83D4E349F87B7154AFD928
:10091000E1EF5355B8E7FE3F0488AE8C031208514F
:100920007465E9EC682459467841D713376D62C382
:100930005B6FDCD2EA54D2E389017E2BF780071487
:10094000D0E51538608C7003042936BA5E14347211
:10095000F6E8A76F82F42D73EA473A676AC0F02F72
:10096000F14ECFA88A1CB9D8FFEE1FBB59D0D6FED6
:100970003F6E6E5255CDDDA8AD72559570E3B6E968
:10098000DDD4844ED9A64B0B65A52B6D2E4D42B6FA
:10099000ACACDB12495DBDF21E022D6C3530A0728D
:1009A00046044E51AA423500400133493A605AF19B
:1009B00032966C2C2D5DDA9C63219FE62F5B294DCE
:1009C000BC94AFEDA534F172B67494BA82C3FECB79
:1009D00059469334E52B57E9855AE2C7DDE50AA766
:1009E0004BA7FF07613D5698D4B6E6A58DC7A80171
:1009F000C5DA332C970612D94FD96D30A665DF7949
:100A00004B8B11CFE0AE29CD4E5D38EAF5F464454D
:100A10004784CAE65DF59601CD976A40031A285DC2
:100A2000D0DB61EC7DF77B3C5316DB9AEAF52E6B4D
:100A30002D6A4346BCCDB33DD9B5DA70DF72E79479
:100A4000EACD9DDD9DBC73A928354F1241E196D4B6
:100A50003D4D24A78A94F8FA377CCD767850EAF891
:100A6000FD3F0ED85CCD032B2AD9D4232BADB42661
:100A7000578F58B2B2565C2D63F6CA5A36F5CC5928
:100A80002B6B91B5DB42B7BC5AEA34575DCA62683A
:100A90005C55B5ABA3A20913A765A82A9853568F36
:100AA000A9B23019DDB3A622CBA4B4EB18B3EA90F7
:100AB000922E6D0DBEC3523AA723C40A4BD95BAE2A
:100AC00050323CA473F8420B3793D5E6F335DD95ED
:100AD0007FABCF87F234DEF7FF0CF8AD540306F896
:100AE0002DD501BF9439E0E7320BB4AC3B25755FDF
:100AF000BD8A110D3963F5284734E0EA4DA31A4940
:100B000091BB568D7A7845D97CB29AE19C78E2F116
:100B100069860992B1D7A76E2ED9C75E9FBA84E4C1
:100B20001C79BDAAD4C4B279CDA85397F0A63CA332
:100B30004B53C39AF28C31550B1DEAB3F6143D2D7D
:100B400035CFD9B31BF3D03EEB2C7ADC53368F2B49
:100B5000C5D6707FD59E14DBC27C55F9724C2FF13F
:100B600097E9CF6AB5C276963F87D2D258F9FFA2ED
:100B7000D53938CAECDBA54CA1985AB9F2D3476FE6
:100B8000E969CA4EDD89570E693F4561D995986577
:100B900067256B86644CACF5E254CD867AD0E63599
:100BA0004CD702A57BF6B0A7BDACB5AA541DDBB2ED
:100BB000F6ECC3D36473D963C82CD5DFE90CA13339
:100BC000D8F2E6335EEE09B6B254DCF8E7FF010C6A
:100BD000887E8C02A50A31DD5CB2AC265BCF4CEE80
:100BE000BBBBDEA7CDA8B4754D1CB7D1D528EEE6AA
:100BF0005B767B9A1AC433F3F16D763FE7B6B6ECB9
:100C000012919BF28E4011CA5D443680007A2F53B8
:100C1000402D2414F87F0A2856B9A545558449CC9F
:100C20009366D719264B4E96DD44BAAEBED9CC108A
:100C30002842B98BC8066080F1E9ABCAA623D43636
:100C4000DFE18C5574866B9FB167BDE1E6BBDB9736
:100C5000534588CFAEDFFF036BC8E2B2423ADFFAFA
:100C600016274FAE7DC417B72C45AFA4B66D8003D1
:100C7000D80CF0A79B073CE080EBB5113845A90ADA
:100C8000D50002347565B6A6AEA2346EEA8B9B24FD
:100C900013A5ADCDA9C886F3CE7E8E6DC9CDB05A51
:100CA0007ACFADEEF54C7789833AA9377FE12FAD46
:100CB0004887B3FC3F662D02624BE38EA5EB1077AD
:100CC0006EB3AA2A2A3974CB2A0BCBB2E4AEAB4C52
:100CD000BCDB9CFAB62A8A2933EE93EAA0A6C4B9F3
:100CE00055E892A854A7C46E1832CC542DB7B5A9B4
:100CF000725351BCAAE2532CB4F52A8A2BB5D2D533
:100D0000AB28A6D4DA5AAF22FB322B4BD38A14DCA1
:100D1000DAC84EA952246B53B96AF051B542E93191
:100D2000C09BB034A7A6D4856FCA5AC20A2EE66B00
:100D30006789C3B4D82F5D250DD352DFF414DF4487
:100D400047FBD25372A21E75094F898D7CB4E7FF11
:100D50000166313C7C52E3C469F585578651AAD3BC
:100D60005675A1699D6F7DCA6A57236DF5CD57D120
:100D70004B50782CDA75694677B4CEDBB145AD08B7
:100D8000E52E221B0018D03C91035A09B18000B215
:100D900013FE7F615A90BAC0D7A6690019856ADA36
:100DA0009ACD24D9CCCB2A467666F5373B9BC948E9
:100DB0007B50D48ED9BDA8756BB362EEF4B8B5ADD7
:100DC000FDE81BAFCCA2CE7BD8FB38B3DAC8D05538
:100DD000FDA96F7DFF1F06E812D9021268E18C861B
:100DE000D4F576C6331AD1744A541E6F262B5BDCB9
:100DF0004293B2ED714D957B8E53DFBDAEB5B0CC55
:100E00002AEEBBF7762653D94A7DFB596E1F2B1B62
:100E1000754DBCE313DEA0A632C8AFFB9318AF201C
:100E20007DFF0F615D964934D20660C7900C8C66D9
:100E3000F615224D37AA6AC82C6DCD28B2158BE461
:100E400035B3687951E6DA9CBE154389F0A2DB958B
:100E500077A7A6664977B19A9E0AD575EBEEF6B0EC
:100E6000C6E683D2E3EB5ED7DA5C48876D9E7BDF14
:100E7000F3894011CA5D4436003860EA8C002CB317
:100E80006D0101145F8E81FF07A39DD69932178FE4
:100E9000668616745FB39AE14AC4F4CEAE46D11D9D
:100EA0005A463A99452BAA82AC0827BE5ADD0C2532
:100EB00042BC7BF5D31761F896DDEF612CCD8A44F7
:100EC000C6E3B1571B6269AFC7999C7B662C6E77EE
:100ED000F66911F6AABC29A487DBE7F4E5141E1A0B
:100EE000ABDD9F627A68ACFA7F08C84A0C01C57412
:100EF00011A0CAEAD1365ADD46DE56554976077941
:100F0000DBC5280AEE6E61FFBDAC0D0245701711FE
:100F1000D90002E8542D00D58405602AB3933567C3
:100F2000669C6B4E56BD9B6ADD3959F1AE6EBDF8BD
:100F300014C5A785E5E25315D59E2E9FCF50E4A694
:100F400007BF596BC53319D8A51C89CE94619B7412
:100F50007ADD13C44BFCE94EA7AE0AA5CDFF030A08
:100F600088A171158576458AFF9BDF6C65995CB712
:100F700072DE9DED7277736C4B543563E4A6EEF927
:100F80003457943963E4865F049834DD020E983256
:100F90005D0312E0C0FF030418B68200D357086057
:100FA000BAF491C65815CA8B479AFC641AAF1959FE
:100FB0004A9DA1FA6464A96586E4E291A7EE99923C
:100FC000AB04E0A2930408909D33039E7165C04F6B
:100FD000290AF8ADD402089CA254856A80008621B3
:100FE00057C04853011836BC65A94BAA4B9BD6C4C1
:100FF000EE11416BDB94EC9436ED6D4B76939EFCD9
:10100000A5EDD94D58EA9ABEB72BC5764F7F14FE91
:10101000D8CD2B7AB2FA9BF288F0AE0814A1DC4549
:10102000640380008EE030C0B253FF0F2B6FB1D944
:10103000D336DFF636B7268508E52E221B2000259D
:10104000AC2A20CFD35245536AA99E4F9B5447B92F
:10105000E4DFC31CC6984565BB789FCB5CD2EA43EE
:1010600067B0E5CD7B389DAD2C1537F1FC7F0A28A4
:10107000306CADC3A7AA70D7D5765D22EE5B57D989
:10108000F9B8A66D5965169BA1DE7BD5996DA5585B
:10109000DED564115DC269CA30255B853221409678
:1010A000260E584A33004BB5ADAE9AF030DFB2C7CA
:1010B000313555E9215DFB34F6AAC63CA5733FFEE8
:1010C0001F06D82D2C0133B767A0C5C58DC8B2B790
:1010D0009617BF2687F95A91F3B01F751945CECDE3
:1010E00071D46554398EDA71B6D1C530E96E69CBE9
:1010F0005C518F156649FB8031A2E67D9D55B6593E
:10110000D8EA710FDECAE59BC7D36592556C2EEF06
:10111000304992B13ABDC30472E7E6F075EBA8938B
:10112000ABFF1F02102C34B446AFC88ABDD484A9CB
:10113000E62DFC461D7B48872A5F557613E9BA7A6F
:1011400097BB9C5569A3AB48D7D5B10F63F7A1E610
:101150002A3B8E650CA95255568DB6926A77F1BB23
:10116000C686B23A44FD9CDB5248D738B9EF7BDDE6
:10117000C3EE7D67B0F48967BCFE1F63A921B43C50
:1011800016AFB684D20A5FB3AAE2DA32F4CD2A935C
:10119000DF28D727ABC8E25B9357AFB2D01B0BEE6B
:1011A000B2CA24AEC3284BA90BAF0E134702A8A6A0
:1011B0004C004D5708A0990C0174EDB1EA22BAD445
:1011C000A9CDAA2BEFD6E0BD6B69AC5A83F7AEB3BD
:1011D000B16A0BDE32F6A23AC27973BDF2FDFF02AC
:1011E00048694D0306E834A285954C78A8D29366E9
:1011F000B1E94D796F7AD39DF5CC012B860660C598
:10120000AB08442000CD108DB626118BE83CE66279
:101210005D3D63F758BB4EF1B02EED28CA74CC9BF0
:10122000B8B769A60E8F66BEAC48C6ADAEFB9A16BF
:101230000EF378FEF3BFFFEDFFFF06784A2D005353
:1012400099B52ADB628B4C34AA12CBC26CF1188A96
:101250009EB094CD6B2A724A8BBAAC39CB6D29EE15
:10126000D2D668AEA5A94BD983BBD4C12E6D8FE170
:10127000CC16B39423D95339EC53CE5C06FD304BD6
:10128000B9725DB4C3DEE9CE65C18EFB86BBACC06E
:101290000A691B9ED212AAB55378F3336EB14CFF84
:1012A0000F0C28302C45439A72D8EB9DADBA0B67D2
:1012B0006E7F3D9AA11DB9F50B02A72855A11A1002
:1012C000D65C3A352C661AA2757333A7A90F51D292
:1012D00054DDB63A276A4ACBB6CA92C82C6CED2ABE
:1012E0007B54D4F2D7A31ADE50261EB77A04059990
:1012F0007CDCEA190DA8EB76AB6630A0AA59AD1AD2
:101300004140AA67A5AA7914AB9EFDFF0C50D6AC4C
:101310009451AB67609F5AD6B60E69B4AA5293BA7D
:10132000E4C5AF0678C655013FA528E0B7520D18B1
:10133000E0B75403FC52A6809FCB103845A90AD5CC
:101340000030C0906E02D85CEDFF0104E8DE1D01A4
:101350004BBB12607A77010CED368AEADDDC64CD96
:101360002A6A344FAD25BB5C55CBE629BD64D7ABAB
:10137000A9C53CA4EB885635B6745797BAD8D8DCC3
:10138000DD59E973E394306F6B2CC142C3BAAEBA36
:101390008514B79C5DCE6E49533D6E3A9B4629F34A
:1013A000780C28AE53031A585DD59319B266F5C56B
:1013B0004C64C89AB1B65896664FC6D55C8BA7BE2A
:1013C0002E57B3C959F166DC3DB7B8D99A72B72226
:1013D000A6DEB5D3D71AB9F4CE46E014A52A540335
:1013E00000143085BA009EAFF87F08684894003733
:1013F000300AE00F1705FCEE6480DF8B0DF06F897B
:1014000001DE544DCDB75ECAE265654D8799D99A24
:101410009557D96E616B5696D584A7AC5E69081B4B
:101420006EB679C4C16F9648A796447D9EC29D5AF8
:10143000D65145187B31C063C40EF8D524007FB85F
:1014400007E077D5D62D114E6A595B57AD70443CF5
:101450001E43D746D6F6682C552AC7C4AAB63665A9
:101460001CE38FC6D65588962F6E47B1219EF9781A
:101470003C559646F8AAF25735AC918BD25F794B22
:101480004AAE66C067A40AF8C9C400AF382BE0357D
:10149000550E30E0B592FF070A28306C745325B31F
:1014A00067AC950D6324118B5731BCA154AC19F571
:1014B00070063CB6C60D91A9CE52283632DD95692C
:1014C000B2F8D8BA6CDA313469A95330E39274A90E
:1014D0002A554D92D397AA46132A4DBFEA1E82B1D0
:1014E00074EBEA860982F6356B18CE1127668D6992
:1014F00038479C5C3C96E91CA173F5D8A733A4CE71
:10150000C5E51841913B1FB7730425AA5C53DE194A
:1015100083306C6B7A8777E48C3DE51DD150CCB776
:10152000A66F382776DD12BEA1833878AFF99A0A04
:1015300014B7CFE9BF24445CF2A6FF2276F3709380
:101540007F057C8FA401016CC8C9801F3CFE1F0C65
:1015500078C695013FA528E0B7520B04E0B75407C1
:10156000FC5266809FCB4E56E524A7B63D451553E9
:101570005ABAF554D96D58EAEA55A7B86EE5ABC723
:1015800098EC8594AD6E4BB49752B62A6C316C983A
:10159000DB46F3F8B269E61BCDE36ABBA92F12AFB5
:1015A0004BE3C1DE8901435472800314A0C0FF03E2
:1015B0006E4A9C624AEB84A508D22E699296AA488C
:1015C00033A5699A8B248F90A663AAD6429CD7AC88
:1015D0003E1BCB525AB2DAE83AC368CDAA42DEF0DB
:1015E000E02CAB086D3583B38C32D4E12AEA338624
:1015F000D89B3A69CF58736EEAA2DCE3CCD5785217
:1016000073B533379348D914AE525C3574120386E0
:10161000A8E400070830D404011A1FFB7F6C657E24
:10162000D3CD1C8B83BA4B37B3C30E5636D9DD618D
:10163000D8759C34A1AE6B4972DC83D6AEAEDAD6D7
:10164000707EB3BAEA5CCBE3CE1A9A6BF1B0C76B8B
:101650006EBA39D25EB5B3DAE4F49CEDDE96C3839C
:1016600022B1019E7155C04F2906F8ADD40201F890
:101670002DD501BF9419E0E732044E51AA4235003E
:101680001430A41B033657FB7F0AC8B3C001B9341A
:101690008F3C37B1284EBBEA34C4B3B8EDAA53E748
:1016A000B032F7ABCE83D32DDDAF3A17B5D0ECB661
:1016B000AA625246F34AABAA71699CCAAE4A82BB7F
:1016C000D85223708A5215AA01A08021DD18B0B922
:1016D000DAFF030CC8A33900C5963BA0734F034C37
:1016E000ADD5B2CC6C42B8CBCA1AE7ACE4B62B9FEE
:1016F00046C282B6AD625A370ADEB68A19DAC169C5
:10170000DB2AA62B8590ADAB9CAE0453B6AC72D849
:10171000122CD932AAE69AB865CBA8AA6DD4952E18
:10172000A52AB6514FB2A5AAA44559F1FAFF636F95
:10173000C47A1DB5ED6137BB6E7562D92DECBF560D
:10174000AD09BA328C13C7D6ED4D858699E33EB705
:101750002986902C76DBE69895BB384F5B7229B4CE
:10176000516F7DAF47B973718C313FE1C9A950D634
:10177000FDBA2757C56ECDFDFF02C8D95C032D8A7F
:10178000B1304652AFBA86261AF6779BD3D5186881
:10179000695963EF805F5A2D60010B68C003AB6E1F
:1017A000DE252D17DFFA36BB1D53B16E235DA75D15
:1017B0002392B9A7627F2050847217910D00A080F8
:1017C000A5330CF0B327025A4AFD7F6A15715CDC21
:1017D00023898DD536B58C2D36DAC6CCDD915AB934
:1017E000BF51C7CC69766AA612D2B6CEDB6B0FCCDE
:1017F000BAAA102EBC29ED2AA25BF3A52C2B4FA967
:10180000259ABCAEBC74D3F070D68AE4C48A3DEE8F
:101810006A9B57358FD46BE83ED82216AE71F820FC
:101820004D5FB4E6E183B47CD658460A94F19973CF
:101830000947AF289D16341CD561A5AA13736543CB
:1018400015E271D2950D6772D84E77B15CCEEEA4D9
:101850003C2DBAA45AE5F274576CA9ABFE1F66B7CB
:10186000527ACC9D84DD4BA936771296C854272C2A
:101870005E1A8A10EEB478ABE9D14C4357AFA22779
:1018800057F158B5D29182CC73F14A4676B4A82567
:101890002B1ECD50BD66AF782426F56EBC630214B6
:1018A00018D6FA63D3D439E6AABB5736A9C5A76DB3
:1018B0005ED9AD979CA1B9608B587DC6EE922D7C08
:1018C000CB99BB29D6F2CD7719EBD4255CB6796CD0
:1018D0003D2669F8AAB4576314930BD3D993924564
:1018E000AE49F7B08132B938DDCD28E6D4A2F43460
:1018F00069D85B8BC2DBAB907BAD366FEF22A6D590
:10190000F8FF016688823ADDE384314B6C0F4F9C0F
:1019100086AAA03DB5F1EABA3371B559AB1A36556E
:101920004357AF72F8524DDDB2F29192346475A90B
:101930009B318A944AA31E3E414A56AFB659C3080A
:101940005FBDBA6A9CD37C959A9DF2288F06681970
:101950004CD8CC6C39602893005C19D6CA6A9D5C5F
:101960006BD1188A31C9A84563CB3A382B1795A794
:101970000495D0995D9EE25543E77579B3350DCF57
:1019800055EECB5E2D3836893F073363E9828060A0
:101990003508505D2A02AA4DFB7FA54F7AD33C5AE9
:1019A0008FAEC8A970EDBDBA2A3BC3D98F006C4A6F
:1019B0002140D3CA0818C20401C3861160DA4C055D
:1019C0005453DA9C5816EDC8EB88E24CECC1362330
:1019D000C865D117BAB420E5E46A8A53A2AC0B7388
:1019E00038C9C8B268CE9224335B45B1A911B66A32
:1019F000754D9698C7AAD63791EC12AFC8D1B18869
:101A0000972576C0962201F82E2C015399ADA17A24
:101A100013F57ABDE6AE43D47DCFBABA0E51F7DDE9
:101A2000ED6AB694DCF7B4B75A5709DF9DBE62DCA5
:101A3000D475B7FBAA5533E73EE22BDC5D35FC9845
:101A4000AF790F0F566DBEE1A6AA42CEFF03621119
:101A5000BDD83295AA99D7268FB0AB263E9C2B4D88
:101A60009D1AD574CA306561744D253298B7360C0D
:101A7000714BD3BEEA983ACCADCF2A921F6FB12DED
:101A80002B4F7EACDC36AD38E7D470DFB4E2522C9D
:101A9000543D5328B2A4F07257A55EAD83D9642398
:101AA000607B93088C7E441772F3DB869285AD7D54
:101AB000571B6B1EA60CFDE52C53315AF3A63B3782
:101AC000A16CCDE2EE9C8DDD37E9FF03A35BCE1860
:101AD000239FAC767913887CB2AA198C2172F5AA5F
:101AE0005A50D2B0D5A97652B253AD952672D51AB6
:101AF0008DD6DA24C522C25EAB93D6B054A5AB888E
:101B000031CD9392AD3CDB5659F6B6925C836C3086
:101B1000EB0A4A5DC645AF23A853C8C2F2AA243BCC
:101B200012D36EEDF2B30C99DD4B00B6133AE5D447
:101B3000A6AC91E754C3A4A1E9B6D34E1946A1FDC2
:101B4000463BB98A8EB4294315C2931CBD8C45B05F
:101B50008D71BD366DA6A6A2690DF08CAB027E4AD2
:101B600031C06FA5161855372EEAFE650C43BB50E1
:101B7000FA96364E9382E57BDB3294336EFC19DBAA
:101B800074C158B1A6ECCB1743FA9A700C6F60552C
:101B9000ABFF1F0A28306CD4C75419AA9BD5346BED
:101BA000CAEE6B56DDBDA944AC59D508C19CB17ACB
:101BB00065332472E7AC958C64E0139557D4BD501F
:101BC0008D451951B39861AE64A4CD609485D290CF
:101BD000474135EAEA5A734A99A03809C07642A3C8
:101BE0009CDA9435F28CB166250DDB3C869A4BA0CD
:101BF00035FB984B72E2B36C6DCB43C847F2A5231B
:101C00006F216FCE168EBC892BB56F38CB32D29632
:101C10006CEE2CDB485BF2B9AB2C112FEE1DEE52B3
:101C2000072543FBFF030AD85C4D03258DA9245AE1
:101C300052B62285311FDCD2F2B44CDBE5CAC85261
:101C40000BEEA6C72DCF5369436EA5BA94802AAA7E
:101C500065FA1C883623511BEB30F4B0366BA85163
:101C6000243DD6ACA184444F7FD4E6414670622324
:101C700002A72855A11A00A08021DD18B0B9DAFF0B
:101C800003ACE77EC2D41CAB8DC731B5B0AD769145
:101C9000D68D2D71584D596791B56BC8B23D9CB624
:101CA000ADA1E9E4487EB3DA968D2D6DF5AA7B32BD
:101CB000D2CCD5ABEEC9513317AFBA87008B5C3CA1
:101CC0009BFF070888DC950155862AA0857605D4F8
:101CD000904E0033A94719BBB49B7B5B55C8DEE629
:101CE00091655529B4A5D9E255E7D01AEEB35797B7
:101CF000536A78CE69538A1E1AD5281C59892787BA
:101D00006D7717251E6299113845A90AD50050C074
:101D1000906E0CD85C0D815394AA508DFF076979A1
:101D20009C4CDCB296E5394D43F66A8009281CB01C
:101D3000098A011E461D53D11666FE664CD944A47D
:101D4000E99BB124DB19265BDA12E38499BE69674B
:101D50003493E1B2A69DA15418C7DC76855469126C
:101D60004DCB154BA5B1352D7708592ED138DD490E
:101D700079B56A9D74572B916676D3D3BC58AAD98E
:101D8000494F5666A51627BDCD8A956A9CF456CB59
:101D90005EA251D29B5DB15B2C4E5F4916A655FBEE
:101DA000FF01ADCDBE452D5B8FB6C87257DBD4EABF
:101DB0000EBC8DAC6BA92790495677A51950C75812
:101DC000D2ADA6882C53DEB2AAA22A2CB8CBA87317
:101DD00068B696BC6348A9305BF2943597802EDED6
:101DE000538E1A0665244F7A6A6E94E13EE96F3E7F
:101DF000892BF223708A5215AA01000A18D28D018C
:101E00009BAB21708A5215AAF1FF0ED82E3500CB5C
:101E100075786004A91865F1EA95E46E9C4B7956D3
:101E20009EAA731C751965CCA1B5B8A6D5D99B64BB
:101E300052D4D6676B92CD71D7904C9B8CAD195311
:101E4000566DDAF6BAAC494BB64A9CB1666F96212C
:101E5000CDC69E79A79576196712531EDCB59C51A5
:101E60005EAB6BD7F4077DA56AADC31FCCB788B74F
:101E7000717F10B76A9A36FC89F6BA4B5AF7473920
:101E800013C179CC5754678AB8F97F0E98A1C40161
:101E9000DD288F74846473AF75EA1A9D2A73F16923
:101EA0009A2FB6B2C7A7AEBA38DB6F9F2AD9928EE7
:101EB0009ADACA66295B4A956B129768D15A0678F6
:101EC000C655013FA518E0B7D25126351EAA8B672B
:101ED00039AACCAF44B5CBA80B9909962CADC964EF
:101EE0002699BBB436919E22CE9ABAC4AA1B2C4B1B
:101EF000EA0B8D0C23B7FF0F088844C500C5B91A3B
:101F0000A064B3D1A52CA5C56B5697B3BAA76E59DB
:101F100063C9AE11BA652D25995ADAEAB636EB2AAD
:101F2000E12913B0AC6B0266D94CC0CCDB0E684122
:101F3000A94DC527497BB6B2D6348CADFECB518EA8
:101F4000B315752D571E4ABEDC25DDB909C54A9665
:101F5000F0E4C39C255DDC539E7225A7716F79A9BF
:101F600069ACF4FF01AEE83998BCD68CA219E598AB
:101F700098B48A6E55BCA3D62A9B36F5F259AB6C41
:101F8000962A5CED8C2A2BAD108E93AA6CC595B267
:101F9000A1EB96493333C7A99F2E3342143BA0B916
:101FA000F65126576A4D5946975CA9376C497DB062
:101FB000EA1554B7F4C94A9452BDD5149DA6ADABE9
:101FC00057DD54A88D6F5E5577CED6BE6A153D2875
:101FD0005BE5C2568EAACCE6AD1330725B0266E9B1
:101FE0004EC04A1B09E8A57D152DAA72D8E655B743
:101FF000A026E1AB5B530D76AAC42975353866E29D
:1020000064D45573A6489C51176D6E1E8DFE1F2219
:102010000B34A2C29CB08C77970877E256DDD4D2FD
:10202000DC499A43270F576F6DC89D9343F38DAAE0
:10203000FA540B5DB3AAEE9BB9E4CDC8A66FC2D229
:1020400035239D71085DD68CBC6761315D5DDA69B1
:102050005C482DCD68AA0B76F327A32FBA244BD664
:10206000B43199751FDAD3C6AC2E74B14F198BB841
:10207000E0A33E65CA664D8FFAA439C79658CA9345
:1020800096949A63395F58634FCEA5BCFF0F08182A
:1020900055CD01D3A90560E876079458DEB254D532
:1020A000ADCCCDC873D3B0E22DA3CAD5ADDC5EAF45
:1020B000AA9A156F59BDEA1252CB6D3602AA0CE3EB
:1020C0008002BA092D55C9EA2E5565CC259886E5BA
:1020D000ECB1D4A09256ABCA56A36055AE44E014FE
:1020E000A52A540318D052B0026A0852400B41048A
:1020F00088DAF0FF0162578D2DDDD5A53D363677A4
:10210000773696DC3825CCDB194BB0D0B0AEA76B58
:10211000DE35CCB69CAA055767DB92AA6AC8827DD9
:102120000BEA3CB7B0AC8604E8C0AD8D2D8898F5BD
:102130009DB10CEF24E16BDA3E7D12867F69D7F406
:102140002D10B6A55FE59921112B5ED7EFFF01A5F4
:102150004DB2D784BAB42ACA5916DD3ACAC46785C3
:10216000A5DF2A2ACA75E56C2DCF28279CBD2170D2
:102170008A5215AA0190A2AECA5CD5F1CAAB32AFA1
:10218000A0CEAB2C3ADC4DBE8CB2380D919CD38ADC
:102190006E48C72C6E299A641DB3B8A5AC5C74CC8C
:1021A00092962A6B7397ACFDFFAA90D5AD559DA969
:1021B0005694D40A97AB7A399CBB445DE8FD143D34
:1021C00053F7AD095DABD4DDAD3ACB0B2FE9BCEADB
:1021D000A2CFBC74D5AAAB1D89D2C7ABAD21A9D201
:1021E0001F8FB15AA7A97A548EE112BCF26538BB91
:1021F000678AEE56089CA254856A008003A6507731
:10220000C0F31504D8CAECFF016E4CB88BB5DAA642
:102210007523EA244B1BD60D6902BD5D5936A249D0
:10222000B47665DC88C73196ADA1F18A30D9B2BAEF
:102230002EDBC274CB6A9B294DB335AB6BAE252D1B
:1022400056AFB1F8D4B29C23806A5205D0752803EA
:10225000BA29E50002A72855A11A000A18D28D0153
:102260009BAB21708A5215AAF1FF0CF8294501BFDA
:10227000955A2000BFA53AE0973203FC5C56F26AFB
:102280002A202CF9C88A2FC195EC23CD319997B318
:102290008F34BB125AF11EF2E442A5C8A9989C499A
:1022A000D508376D29265552BAB6B558170F7FDDB8
:1022B000CE6C5DC2F3D7789A4951B3CEE5AB3AD92B
:1022C000CC7695BFDB7615F667805F530CF06BB26A
:1022D000037E4E37C06F660AF8ABD9007FA629E0AF
:1022E000B792FF07662B2ECC9812BBA34B7713B780
:1022F0005D8E6A5C43ADF5EA723077ABD9AB293EAF
:102300002CAC16AFA6F8B4B45ABCEA9ADCCABAF63A
:10231000A86B110FEB50089CA254856A8001660CD3
:1023200056C089A5069821B94DCD2B6AFBA6363734
:10233000EFC4ED7BDAD6ACB3B4F6697BB52E56D2DA
:10234000BB1CD984454AD37266551E2EF1CAD5945A
:102350005B989A297717AEE11C253D4DA6858B9990
:10236000FF07AB1FC1C93367AD7A9A649D98B58AE0
:10237000E18B357DD6CABA098E8CD92BED8ED3D49C
:1023800013AFA4194A3773B592AAA8CCD4754BB32E
:10239000A07609D72D4F82CBC2138F625812B54A4F
:1023A000E580C258563F63B930EB597D0B2A12BE07
:1023B0007A0DDD8652D8D6B5769DC6A15BD6367528
:1023C000B804F72D47B3E4A566B79C45B29758D437
:1023D0007215C5D6A271EB1DEEAAB13C5C4D789A80
:1023E000C6080F25FF0F0A2830AC3543858958DE13
:1023F0005167ED6EAEAB579D448726771D4DA253B6
:1024000016EC6D36A5F775D493BCB525B4E64CCE65
:102410009AB6509B2AA95F3AE27069C73E698BD38E
:10242000B903FB862BD5C46CF6939E5C12AAC46FCD
:102430007AF234F256BFE9C9CD30CAFCA527176538
:10244000ADE813DEEC44C363B3799315F1C8D5E965
:10245000BB24445CF2A6FF2276F37093FFF47F1F47
:1024600061C2CC14F03C9206FE1F0AD85C4D0323D7
:10247000A8D6342C1AADAA84B4485FB29AAADBBDA0
:1024800075CD6A9A6D8DB6D5AB69A5A83C1A810247
:102490006A2833C04BE50E78CE4C01AF86A7E259CF
:1024A000379670D3CA6E9DD4ED4DABBA36D48A3709
:1024B000AD1C4ED1AB16B7727881C89A5DCAE115D2
:1024C000A266512A4650F098C5A1688A79B243A9FC
:1024D000A27B45318FFDFF08885B4A00396796ACC7
:1024E000A47011F5B2AA1225C4ADCBAAAB2CD1B4FD
:1024F00035AD6D22C4C53B05E0593105BC97CC8094
:102500001D1915709249897FF00C55A7AD2A3453D7
:102510005CD6B4B6211F0BEAD2DA8A7CDCA84B6BFE
:102520001BF271C53EADCDA4CA595AA7AEC18C10DD
:10253000C993D64B42C425AF02BE4712C0869C0A3F
:10254000F8D9FCFF010CF88E59007F0629E03747C7
:1025500003FC1EE2805F4302F06BB0037E155DC991
:10256000A4E6E29E65954D9473E89A55775ACD6E30
:102570005B577D285587381B75435D6EE266954530
:102580004C9859CB55363C1EA6AD5AD514466BB067
:10259000297595186DA62CD54560ACB1F3D28CC0C9
:1025A000C626495B555D08657419654981DADC65A5
:1025B000942535CA729E5696DC2047795A597C2359
:1025C0001FE709798AC25BBE2A0D25288F57ADFF08
:1025D0000761EECA443B63ADB91967DD6CB5BA1645
:1025E0008BA46DF36A5A1A92E12DA32A795096367C
:1025F000B72AFB453DDC9DBA6407A2393102A72802
:1026000055A11A4080625E0590DBA802726B1F59CB
:102610009E14A99669D4B9B197D9E6D517DB622380
:102620009BD754D5A8AE6E5E7357A332B279AD4D29
:10263000ADEAE8E6B596509C61AB0C504DAA01BAE4
:102640000E654037A51C40E014A52A5403C0004382
:10265000BA29607335044E51AA4235FE1F000000AE
:1026600000240027002A0000000000250028002B7D
:102670000000000008000201000003040700000041
:102680000000000000AE36BED29DB3ADDAF84A7746
:10269000CEB6EB5DEF7AD43A56BA73B652F33A61DE
:1026A0006269434DEF86B1398EB5AE55CDF2470A1A
:1026B000DB79AE8EDED64DD6AC3A7A5B375973EB0A
:1026C000519B1C6BAA6D5A2D7BAD89A54D359FBDC5
:1026D000269E36D4F46E189BE350D3BB616C8E1FDC
:1026E000AE8EDED64DD6AC3A7A5B3759B3EB5BDFB4
:1026F0007AD7AB8EDED64DD63CA64EC6954AF68E20
:102700003A19572AD9BBEB5507EEC9A55D773D6A43
:102710001ECA2D7451AB596C0FD3050FAE4E3CBA87
:102720004CFC9E3AF1E832F17B6A27ABD2C5DBA9BB
:102730008DAE2AC76CA316A1368DB2B69AD5DA1023
:10274000C9546ABABA932CD503A6563D5BD4BAB61F
:102750005AF56C51EBBA6A3D3D53A4EDA8CD914AB0
:10276000D1CCA33647B245B3B4DA6EAA746ED16A3F
:10277000375D74D0E703A616A596D4BBB45A945A15
:1027800052EF326A51B34C35DBAA65F34C91B6A3D4
:102790009653AA4433B75A0DAA746ED16ADD5C749D
:1027A000D0E703AEF6C63392F2AEDA1BCF48CABB0F
:1027B000EB5BDFFAD6ABF6C63392F23EAEB6A6C6F8
:1027C0004DFCAEDA9A1A37F1BB6A6B6ADDD8DFA925
:1027D0009349D7F2C6A7F6C529BDA3AC3A1671F145
:1027E00059B2EA58C4C567C903AECE455C7C96AC05
:1027F0003A1771F159B2EB5DEFBAD4C1C398A52A6B
:10280000573367B7A4AA436D946B48387DAE8E45A5
:102810005C7C96AC3A1671F159B2EA58D4C56AC9D3
:10282000AA7DF1108D25AB763593C5DAB45AB71A67
:10283000116B9B6ADE67593CADABD9BD6209A7A19C
:10284000A677C3D81C3FAE8E455C7C96AC3A167119
:10285000F159B2EB5BEF7AD7AB8E455C7C963CA628
:1028600076C3C947FCB7DA0D271FF13FEB59CF7A82
:10287000D6A376C3C947FC3FAE6E29992BD6ACBA16
:10288000A564AE5873EA9A8CB57BCDAD575DAB901D
:102890004E3619752D42DCD57AD4B5087157EB0741
:1028A000AE2ED55C74DAACBA5473D16973EADCD459
:1028B000D4BACDAAD35035EB2EAB8E5BDDCCDB8CFE
:1028C0003A5C09376BD36A7F28D3BCC903AE4E3D4F
:1028D0005CA5DAAC3AF570956AB3EAD4DD45BBCDB8
:1028E000A953F710A9D6A74ECD822D9BAE3A760BF1
:1028F000F69CB7EAD82DD873DE03AEAE3904D2BB4E
:10290000AFBAE61048EFBEEB55A7EA42A55D571DEA
:10291000873996741FB59F2632927FD4AEA9EA6A92
:10292000B607A6EE4919AAC78CBA2765A81E33EBCD
:1029300055976C825153569D8A1B59CE5975A811D3
:102940002CBEA4D5BAF5085BDB54F33ECBE2695D3F
:102950004DEF86B1394E35CB1F296CE701A6EE4904
:1029600019AAE78CBA2765A89E33EB59EF7AD6A34C
:10297000EE4919AAE73CA676E6D7C8E78DDA995F53
:10298000239F37EB59EF7AD7A376E6D7C8E73DAE5A
:1029900076ADCAD56AAFDAB52A57AB7D6A57AA4277
:1029A000ADF6A96D9A36D3C6AB3669C64C9A8C5A29
:1029B000F529516D5D6A71DAA8CDC903AEB6B1D7FC
:1029C000319AAEDAC65EC768BA6A17EB9C22DDA9F7
:1029D000BDCB4DB6E6A7F6213B559A9FDA578F0C33
:1029E0004E3E6ADFDD32B8E903AEB6B9C7B813AF01
:1029F000DAE61EE34E7CEAD8BDC4DBF1A953F7E268
:102A0000883AA7CEDD92329BAC3A3509C9AAB3EA1F
:102A100090547C63F203AE0E2E5F42E7AC3AB87C72
:102A2000099DB3EB5DEF7AD7AB0E2E5F42E73CAE6C
:102A30008E2DCAB89AAC3AB628E36AB2EB5BDFFADD
:102A4000D4A145AA569C55C7EA655A711EA63622DE
:102A5000469DBB8CDA881875EEB26A2362CCC9DF5A
:102A6000A80D8F53537FA3363C4E4DFD3DAE8EC611
:102A7000379CBBAE3A1ADF70EEBAEB5BAF3A1ADFA7
:102A800070EEFAA60EC6954AF68E3A18572AD9BBAA
:102A90006A673DB9B4EBAA8DF3E4D2AEADE6A1DC32
:102AA00042173DAEF6B23A4DBDADDACBEA34F5B6DB
:102AB0006AABBACAD9EFAA65AC6A47EFA566B53664
:102AC00044323DAA563D5BD4BA965AF56C51EB3A66
:102AD0006A3D3D53A46DABCD914AD1CCA5B69B2A9E
:102AE0009D5B3CAA16A596D4BB945A945A52EFD239
:102AF0006A51B34C35DBA865F34C91B6AD9653B231
:102B000045B33CAEF6C63392F2AEDA1BCF48CABB31
:102B1000EB5BAF3A3A4F0BDCF6AE76B6329DB3AE16
:102B2000DAD9CA74CE7A6A9FC2426DF5A96348D1D8
:102B3000F435A70E2EC423AB3CAE8E455C7C96AC20
:102B40003A1671F159B2EB5DAF3A1671F159F2A62E
:102B500076C3C947FC8FDA0D271FF13FEB598FDA97
:102B60000D271FF1FFAE6E29992BD6ACBAA564AE26
:102B700058B3EA9A8CB57BCDAA6B15D2C926ABAEF9
:102B80004588BB5A3FAE2ED54D79DAACBA5437E5FD
:102B900069B3EAB8D5CDBCCDA8C39570B336ADF650
:102BA0008732CD9B3CAE8ED95DA326AF3A66778D3A
:102BB0009ABCEB55C76C2991A347EDAA8665977E11
:102BC000A6AE3904D2BB8FBAE61048EFBEEAD43ABB
:102BD00020457DABFD349191FCAD764D5557B33D0D
:102BE000A61E59097C578E7A6425F05D39EB598F02
:102BF0007A3665B05EF5A676E6D7C8E78DDA995FD6
:102C0000239F37EB5D8FDA995F239FF7A60EBEDB1C
:102C1000D5EB8E3AF86E57AFBB6A176654A2DEAAA0
:102C20004DD81189BAA3B6669ED5E63CA6B6BD229C
:102C30008D9B8EDAF68A346E3AEB51BB6D51CAB574
:102C40005BED0FAD49476EB55FD82999E001AEB68F
:102C5000B9C7B813AFDAE61EE34E7CEA582383AB5C
:102C6000C9AA737735ADBAAB2E5DD4ACAA3EAEF629
:102C7000B947C59BACDAE71E156FB2EB5DAFDAE77B
:102C80001E156FF2AE8E2DCAB89AAC3AB628E36A1A
:102C900072EB5BAF3AB628E36AF2AAEE5599AD67DC
:102CA00097BA5765B69E5DEA5E95D97A76AA475679
:102CB00002DF950FA6F6B23A4DBDB5DACBEA34F590
:102CC000D66AABBACAD96FA98DA96A47EFA966B50A
:102CD0003644323DA67643B9CABCB7DA0DE52AF3CD
:102CE000DEEB54BBA15C65DE1FA6F6AE82C3538E3D
:102CF000DABB0A0E4F396AEF2A383CE503A6EE210B
:102D0000540CF2B5BA875031C8D7EA1E42C520DF4D
:102D100003A64E3E4BC9E78C3AF92C259F33EAE4D3
:102D2000B3947CCE03A64E3E4BC9E7B43AF92C25AA
:102D30009F33EAE02C9533E903A68EC6379CBB8E01
:102D40003A1ADF70EEDAEA687CC3B9EB03A6B6463E
:102D5000AB0CC3B6DA1AAD320CDB6A6BB4CA30EC1A
:102D600003AA96A59CCC37A65A967232DF986A5968
:102D7000CAC97CE303AAF622BA1EE096DA8BE87A87
:102D8000805B6A2FA2EB01EE03A6F6C63392F2B681
:102D9000DA1BCF48CADBEA602D3CA9DF03A69E41BF
:102DA00015BA5A8F7A0655E86A3DEA1954A1ABF56F
:102DB00003AA8E455C7C96943A1671F15952EA58F2
:102DC000C4C567C903A68E65985BB5B73A96616EB0
:102DD000D5DEEA5886B955FB03A64EC54334128F9B
:102DE0003A150FD1483CEA543C4423F103A64ED592
:102DF0004D32ABB63A5537C9ACDAEA54DD24B3EA02
:102E000003A6EE2D982966B7BAB760A698DDEADE6C
:102E1000829962F603AA1E59097C57A67A6425F0A6
:102E20005D99EA9195C077E503AA76EA5E29539702
:102E3000DAA97BA54C5D6A1D7F583BC303AAF62A1D
:102E40003F585B97DAABFC606D5D6AED6F1CB3CEEB
:102E500003A60E66DB599BB43A986D676DD2EA60A3
:102E6000B69DB5C903A676BEA6C89AB6DAF99A2267
:102E70006BDA6AE76B8AACE903A6CEC39325E3B4A9
:102E80003A0F4F968CD3EA3C3C5932CE03A6F63526
:102E9000C3ACAAB4DAD70CB3AAD26A5F33CCAACA3D
:102EA00003000000002300260029000001020304A3
:102EB00005060700010203040500010203040504DE
:102EC00004040404040404020202020202030303D1
:102ED00003030301020408102040800102040810CB
:102EE00020010204081020CCA126BB839318CF4AEE
:102EF000AD2E31ED3CA72426C354F192648B8A9801
:102F0000CB2B2E34532D0E2F57B30C0D3CBC3C4C09
:102F10004BCAF4F0720F6E4953CDCB532D354D0F84
:102F20002F0FD70C0D3DBCDC4DD3DDC2F072524FDC
:102F3000579BC3AB89BD422D0FAF5AD1719155BC80
:102F40002CC53BD865F28294184E3BC17342323394
:102F500015454F79526A55A6A3FF07C36C86B32760
:102F60006D0FA748994E553CBC2265364DD1F032C5
:102F7000D3BE34DAC3EB82E2DA6535AF31F26B9758
:102F800095BC86D86F82A6730BC69E7299CCCB0275
:102F9000AD3C9A1060AB62052C378400A973000029
:102FA000FE1F02B83A8C01DFA473400147B92F33EA
:102FB0003B735F537CEC9AC563D5D175AE5BFC6403
:102FC0005C358791F18336B56855C56FDA452D1CA0
:102FD0002DB738379F603CBC9A85A32566F78A5782
:102FE0001CA96756CA5EF0B216B2F189CE8B922543
:102FF000C72B33CF48B199B4F3FF0ED8AEDD030E23
:1030000038A6D201D3B42CAD6A359DB17DDCEEC4B7
:1030100065D7F1724724B319D9D905704049EA023E
:1030200098BE4201DFA4694000DF95FC3F02E83E04
:103030008C01DD650860984C063493CE80E6DA9A00
:10304000146BAA47D15E56AA6D56CD78D9A91C67D4
:103050000583E1A4BA38EE16869BFA60875B186E8A
:10306000EE8B1D6E61B9693665BA8DE5E53E1CE9EA
:103070000E969B5BAB952B586ECEE53A6AF3B8354E
:10308000847B05A3E336EF9219B486DBB469B4D12F
:103090002A4E659A99CE28D985714C186D6747C616
:1030A0005E534A9CB5E2854526FE7F0C18B69A0110
:1030B000C3750960D80E0930A09BB6A0BBB0AA1694
:1030C0004E82EBEAA9FA59499E59239A273B786622
:1030D000AE4A9C9CE099D32ABD7292EFE688E44503
:1030E0004D7E982D626737F9A137A76C94E4C71E0F
:1030F000DC3CA5831F8BEB520E0E7E2E4EC731D2C9
:1031000079A53A0DD9C4FF0702D82E9C01DBA6335E
:1031100060FB3001EC20128CE4D8CA329673634114
:10312000398998C14D0DEDB02A05370FB4A5AE5CB5
:10313000DC36D0832F4A717B03F73859CDED1EB4AE
:103140006B1435B76B949991D5DC2648774B667133
:103150001B21DB2D8AC96D88FC26283AB721F41F74
:10316000A365BC0238BB3D8EF02BE208B734FF0FDD
:103170000E386E2500A30D3AA037C5A0059E563522
:1031800086AA5E8CA482B2D774312269AD1CD3C1E9
:10319000D0FA282B2D47C31BC2C4AEC6CD9C4853C2
:1031A0009AFF0FCC677542595D3A4F9D3663B75908
:1031B000DC305B5C2361F3E21CF1F098C34B7D399A
:1031C000CA1D2C2FB715EF7079BCD2467C52E5F1A1
:1031D0004A6AB37147C32D39344B2335B77A553317
:1031E0008F59DCA244B5BC66728B64F5F698C14D6C
:1031F00042D42762382F4AB69C8868BCA695F85CF2
:10320000A109867791115BFF0FC6C9715AA292146A
:103210002F6E979C469DDCB04D621B5570DD55BEF0
:103220000E36C13337A9A7511BCF3CA59E44AC3CF9
:103230007D987B529672654BF61AD9CAF5912DA2EC
:103240002A4BF7FF016DFDC65C95D5F5D5027B5D78
:10325000FD512D2AE47775A33AB1FA9B5DEF6A55CB
:10326000332760D4E2D9CC764E739D7B3FFB59AEB9
:10327000550AC1734DBDEA9D9E1512A06B757EFE69
:103280001F6AB1A2A795D2D8250FA32DB27A1CB37D
:10329000DEE6D4456D56CA9A5BDFFAB6BBDBFD1A93
:1032A0008A6F2BF3377B194BD32539FAB96F6DEB46
:1032B00031C45C1EF7AD1FE51CA5485C1ED72B5F13
:1032C000F9FA7FAD68C9C53256DFFA542D357BF85F
:1032D000EA5BDDE64C6D04A6C5EAB984B575233713
:1032E0004F834011CA5D44360028A0E6310F68C004
:1032F00000BF8D79C00316D00007FE1FA1DEC244B7
:10330000C2FC9C6A887009597B8ACA3B3DA4CFCD18
:103310005696C4A6BBF46E59E29DEAE24AD5126500
:10332000BBB3EB51571299C1D96EB7C73135926A09
:10333000C99BC7344C12466C99735FDAD29292647F
:103340006CEE6BD96A22718FCFE52C41D4DD36A5A6
:103350003B19F50CEE13EFFC9AD785C862EE6DBFF2
:10336000FF0766F3D23843B3D82DAC4DBB70B0DB4A
:10337000B00E172C26AED3326CBB32AB1963F721DB
:103380006C9CE5D433B680CB9A9BAF6CE542707FE2
:10339000B3B39DEE7C552B2640D5E2D9F6B14F75DF
:1033A000AB7B3DCA354B1398AFA9577EF397BE1937
:1033B0000B31F3CDFF03A19F9C9472268D760755A8
:1033C00090783CEB599DA2876076DA728B5336A5D4
:1033D000642D7B6EB5FA24DC32B1731FFA1C16AB78
:1033E000C6CAE0B5DFCDA1D4781BB6539774A72128
:1033F000BCE4FF0101D8B6DD012FF43860D5D191CE
:103400004D9784E64B4E36B21067CD19D92C0194F6
:10341000F1786633EB79AF7B578736AF52089E6BF6
:10342000EA5AB77A94734547AC5A9CAFFF076B6E64
:10343000D9346CE6DCF636B7BEF519AA0F2DDA25BD
:103440007B195B4D9AA2E7B81D23A526712A03FCC0
:1034500094E6010F68400312E0000730F0FFABC8AC
:10346000723393BBDCEEB6B7B9F568535CA9A64DD1
:10347000B36B730ACB71D8BBAF7D2F47B6C7F4943B
:10348000379DA934F8539778FD3F0E98D52802113F
:1034900018E9CC4698F166A7271D219992B6DC7CE5
:1034A00017AB2CD22D133BEFAA75CE9447D0EE3A32
:1034B000C4292F613531A250B6F8CD1FFF0F028805
:1034C00026D4006D96B5B82505896C3DD2E651B37A
:1034D000A6F4486709A08CC7339B79CB670E80CAD6
:1034E000D7BD6AD57206B4B5BAB7BDAF735DF391F7
:1034F0008F78FE3FA36DB4BA8DBCADA692EC0EF2F0
:10350000B6AB5D8CA2E0EE16F63FCB39CCB1AC91F8
:10351000E50C8BBFB03BD31D2859E2E94F7BF9E79F
:10352000FF0141EED1C8B316EFEED4C33559C4E361
:103530005BDDEA56BB59ED92CD91B4784F63199E8D
:10354000382C9CCEA5AFF508C7B0C2611E351EF160
:103550008C57BCD3DD4D49B8CE0EF734AD16BCF94F
:10356000FF01A9E8C5D87316CFE20EB7BBCDA9BB42
:103570006FF1F0D5B7BECDEEC65063729858EE73BA
:103580005FDBD662729858AE7BDDD35E457293D80E
:103590008D873DEC61CF709658E1A24DE215EFFFAB
:1035A000076B682ED82A37DFFEF6A7AF21BCC417F9
:1035B000DFFEF667C86AC34D3ADF614D956CA671B0
:1035C0009EB1369853495EFB5A8E0A7A43D94F3CD6
:1035D000C259E0F408F90967033119A2259EFF0FCB
:1035E000011891B9004D914660652DB3B867ED5350
:1035F000F41464114B6E798B5BDEF274C3056AE7D9
:10360000EA3DEC712F6D1FB1002BDFF4A31DB32435
:1036100060D4E27AE52BDFE91E4348A3EBE4FBFF2D
:10362000016E5AC19954B20960492207ECA816806C
:103630005D26C7D0A39278743E552F216AB1FA5601
:10364000B7BAD5AD6F7DBB3D8E75B422367F53CFF3
:103650007EB567966134DB529FF48EDC88E15FF2C1
:103660009DEFFF07AA8D63A8AA66ADB9A8CB08DDB8
:103670007CFB5BDFFA36B7396DB5A315BAF876BBBC
:10368000DFD39ED7DA5C49A52DDE7BDB6B7629AFD5
:10369000C76DEF31D85C1EF7BD1EF548E72889E2FB
:1036A000F2385FF9FE7F65186D902DD6ECF656B7AF
:1036B000BCC5AEC730A3016D2DCE8B3DDCD63C61C1
:1036C00076C5259B08E52E221B0080012B873860DC
:1036D000E5ED0858C00216B0800634408076D3FE6F
:1036E0001F6E3F298D9895CD3D00AB3895E2D4EB08
:1036F00034817AF251535075EBCE76B6D3958D92D4
:103700004899AB77BECBDD8E7196048C5A3CE73975
:10371000F7AD6EF52AD72A85E0B9263EF1F97FABE1
:103720001B6194DDD6DCF174DD37B9E7EAD335B33C
:103730001CE1AF6F77C7B5D4E0569C77DB5A9DEBA1
:10374000988C61C030E91AB0800514306DBB062436
:1037500020010E10A006B5FF07A2599551BA17F720
:103760006A95AB3842E4925DEE6215333B50D692D7
:103770005DAE6AC504A85ABCEBDDEC7677BBDFD33F
:103780009EF63297BEF5ADEDB33481F99AFF070688
:10379000983068E46B84A0E8D3938DEC849E4B6EE4
:1037A000368A190DA8EA71AF7ADFE7B2ADE000D32F
:1037B0008BEB9E8F7CA673E540A85A1CAF78C5DBC7
:1037C000DFFF0FA62FAA055CD68CBCC71670593335
:1037D000B2950BC1FDCDCC663AF351AD9800558B37
:1037E00067DBC73ED5ADEE752FE72C4D60BE26DFFB
:1037F000F189EFFF03652C96AD7B6A9F66E4208D0F
:103800009C73AB5BDCE296B7BAF56A6628A0CED5AE
:10381000BBDBFD1EE638A736CF9C80518BEB52D721
:10382000BCFF3FA0DAA2B23A44559CFAB0BA467245
:10383000DAD1DBAE475961ED2879ED45AF5ADF604B
:10384000F43969AB63D93BD2BC24A5F5B60F80012E
:103850003E6365C05F63129080062420010EFC3F2A
:103860006EF08AB34BEBC6AE36A71A3A5453D6DC89
:10387000EC6623DF582643B4CDEA745D9446F09697
:103880003B9D79982675DBB3D7B6F590A8919FEA52
:103890009EEEE99B207DCBFF030828A64B005556E2
:1038A00023A09A9912E71218C35D5652ED29ACE98C
:1038B000DFD9AEE718D65A12AC341F02A72855A19B
:1038C0001A0008D8269401BF9571C00216D080074F
:1038D00034C0010EFC3F089CA254856AC0FF0366F9
:1038E000A91272429B86A51B900E6D76A6262BDC34
:1038F000A5CF6D4F954DA5BB6E5E45315E65926659
:103900001445AAB4989D5A842A18F69274433AAD85
:103910005C27DD6D98A309F592A4654C4DA48256F1
:10392000973977C768F15DD6DC1D63D44FBEC39D60
:1039300053814EF3899FFFDC5F6692B57AFE7F0C60
:10394000F84ECC003FBB1BE0775703FC1512803FBD
:103950004D57D28DB2B82F5EE9F0CEE4FE786523E4
:103960001852E5E2948F4A10DD95103845A90AD522
:103970000004847C820055DD5A164D87156F5E4B1E
:103980005615DEB2796C59A747DBAA72669D96ED93
:103990000BC3934C7857CC0C7FB51C239558FD591D
:1039A00073A47A62F2376EE2666E08F01D91007EB3
:1039B0007134C01F2906F8B5D400BF171BE0674358
:1039C00005BCEEF2FF04F8C55101BFA66A4003161C
:1039D000D0C0CAAB752DCD2537BBD9CADA540FEE8E
:1039E000D9296B4730D8E380006A266D55EBCA2190
:1039F000B9E4D4DD26A5F9E33DB67538A3315B9A69
:103A0000B6115132D2AA3FFC21CE22D1D72D9E39F8
:103A10000B374ED726E1FAC45542FD85FB7B771361
:103A2000A3278003D02520010A202069D6FF076143
:103A3000CACC385B9AE6A9B6A7EC2AC5DD17DFE247
:103A4000E6236B16C32D92CC72B5D5BA86D5ECB9E8
:103A500094AD9890F47914DE8E533C63230245288C
:103A60007711D9008080CF5805F07B990438C001C8
:103A70000A50E0FF01A28FDA63B723A6A16AB1CB97
:103A80008E34C6A69DAAB3D2EABB37F28845A36D91
:103A90004634256B973649EA947012BA2869822B0E
:103AA00071085E125255A50E784EC8014F931BE067
:103AB000E5760634CF2E805ECB02D08C531B52E1CC
:103AC000B088AC6D88452252D7A4391AE32A4E9AA1
:103AD0008ECA83ACB96E3B8B2E0DE3B6E32C3ED57C
:103AE000C3F6B4AB99344B595DAE2653BD647379BC
:103AF000AA216B77ABE9894AA2251223708A521555
:103B0000AA01000A98425D00CF5730E03B4105FC16
:103B100012A6809FDD14F08C2B037E4AF97F6D6C1A
:103B20006E895B368FA99B115AE933A73117B74AC3
:103B300047FDC6929A8B2F654B6B1CE4D5D82DAFF1
:103B4000658D83AD9AB29523769358CAD7CEEC573C
:103B5000F8D85B3A8B3DC5E77CE9CDBD3086DA8687
:103B60002F978238EC13FEE407ED354BF8734EECDB
:103B7000D23CEE2FCBB99D3BFF3F00000000000080
:103B8000000000000000804A6ACAAC2A2629795049
:103B9000F1AE88AEB42A54335A87364B65358BD391
:103BA000BAE643454449E98632619224AD1C3604A5
:103BB00045E3B6625825B158728A69142572F12915
:103BC000361792AA59AB589C28AB269D627126AF36
:103BD0009E74F2C585AC6AF6C9975694AAC5279B10
:103BE000DE5033679F6C1843CB5C7CB2A244BA6A48
:103BF000F2C9AA32CEAC39272BC62463AA9CBCC911
:103C000060979C7D8ACA525C6276AB0A4B51F3C9BD
:103C1000A5AE2C45341AA7AA5357258F5BCA6E420E
:103C200044D44EC93B7731F1D4A5AE32C9D46B9F91
:103C300021ABC0CC287D8AA21D3362F4299B0CCC19
:103C4000F0D1A7EC2AD1DD469FB2EBC0301B73CA7E
:103C5000AE83426CCCA8AB1209ECAAADAC9264DC8A
:103C60006797AA28E8F07293AA2C6122537569A27B
:103C7000C4690BD7A1B19237AD1CB9C673CD2C4F17
:103C8000D29A115C29426CA99B2276AFCAA31A9CD6
:103C900028AA27AF6A4926CD9E73EA6504396BF6D8
:103CA000A9A757E4A8D9A71A414823979CBA1B662D
:103CB0008B5A7C9A2ADCC4624E00B44E7140F049A3
:103CC0000A486A4D00968D0B40F815058869B4AA1C
:103CD0009036456DF22943EE12F1C9A70C758C3D63
:103CE0006B9D32E475CC8E7C8A183631B3F2CA8370
:103CF0009E268D99A9F0660BD343AB82854A618BD2
:103D0000453266D35D354EAA0777D70A2BAD9F544F
:103D1000C333E2843AF12A5589B5D2E0D6D962E2BA
:103D2000C9435963CB51278F7952C46F9D3CA64A32
:103D3000D59872B214CA4C7DD149532875C9DA2D71
:103D40000D31D425AB1080264B02486FC1F26ACDED
:103D500045546A4BBAF5AAD2C4A39932353CEA8CD1
:103D6000B1AB64B7A87CB6A24DCAABF4E98A562BB6
:103D7000CDC1A72FC1D4ADCB9CBE0473D7AC7CC63C
:103D800092DD5D72CE194B4C0BF539A72F213C34D7
:103D9000E69CA5F888945C728EEAC24B6DC959AA5C
:103DA0004B2FD52667AD2EBD54D79EB3BAF2525DC8
:103DB00073BA6ACA4A75CD59AA6B2B9135A9CA69DB
:103DC00028DC67912AE4D4D2AE88AAE0C7DCB2012D
:103DD000AA82C82C33DB0000000000000000000FA6
:103DE000698E8DCD2295B7A97409B2547FC616830A
:103DF000CDB5EF1A7A182297BE75629308E52E2288
:103E00001B0004E09359CB9253CB8C9AAB68D1C57D
:103E1000C25E9FB2A5220FD972AB5BDFE64E63A9EB
:103E200025B04A3BCFAD1FE9AE7A854EF2E527BFFC
:103E3000F9CD5FFA4A1C92E3DCE92B35A95A72FFEF
:103E40003F0228BDD4ECC1979999AB31A4AC69AEBF
:103E5000F656978AA6A5245F5D6A96EED676B5A932
:103E6000A687FBE6D564BFEAA98B579DE28A872F18
:103E700059558C6DEEB96494D1759466AB5655C99D
:103E8000D9EC8E439D258DB3641143E0E121195394
:103E90000E61EFCEC8C5B6FC3FA92F122744DCA6A1
:103EA000A129180F4D1C8624784534751AAAC471AF
:103EB000D5D8AD2F0ADBCD62AFAE1B330A7BBCEA8F
:103EC0006E4D39E4C9AA9B529592D5ADCDDCDC4B41
:103ED0003E9521CA700F7D1D16A733CAE491DBBC45
:103EE0002C0FA72FEEF0B2DD9DD6A8CBCB71735A65
:103EF000635E2B2632A8ADFA9C193795ACE6F7BE67
:103F0000DC55D39ADFA9F130496A7EAFDB42798D67
:103F1000F94376738A35FF0F08C8461303ABAE5ECC
:103F2000CCB36BAFB69910ABBCB3EAE65234E2F651
:103F3000AA8A7355D735A6F1DA55C3568576C810C7
:103F400063B333B21654C46DF1CA7A5096C825A330
:103F5000E841D1321FCFA256FF0FA989E13C3C6650
:103F60008F31EB0B2B5FBDA662C6A2ECF16AAB6B87
:103F7000AEF647AB6A31B03C178FAE67438B5A5CE5
:103F8000C69E182D6B76585A40F198C66A6FD2209B
:103F9000BD1B1BE04913037C1366801F3D0CF053CF
:103FA00084027E7757C00F660AF8294401BF160BBA
:103FB000E08F34017C6BF9FFA96B21B922669FAEBB
:103FC000C7E1707B72BB5BDFEA56BB5C65CB66C545
:103FD0003D67D7AB6D2E643093EEB1CD3D92B99A6B
:103FE000DAB28E40129A6AEB968F7898B32AB4D3DD
:103FF00048AA2F7DA77BFB0C73715CCE6E5C526C64
:1040000073799A134B8945E96E4942A957FF3FA935
:104010002A4238BA63A6AE0B218D6998FA29152574
:104020006A56E9BB53E4CAC5A3EDCA995ADBB6B6D2
:1040300050772DEE1ABA84A224A9ABEB03EDD4A4D9
:10404000D56E12AAB29C13FD3F01D84133003366EE
:1040500029A058A3920463EEE593465A98A514B795
:104060006D59611656D03565856A5A43B65464C396
:104070009501F15AD5857814B46B7527529ED06D91
:10408000D5836A7B60B75377E66D8EFD4EDB688C17
:1040900007F53B6DA5D911946FF585D58473F6317D
:1040A00016569326F9C79A594D9AF86B67E635A1CB
:1040B000E2B75C8977A7AABFF24439ED2A79CA131F
:1040C000D4968AE52D4F705B2A96A7FCC14EB97233
:1040D0006EF77B7FA92C79CC6FD2BA8AF5F97FC2B3
:1040E000563C7DDC12DB3E8C89BA4C4A96D37595E2
:1040F000126EBD6FB7BA165A583DB303A61476C0F8
:10410000CC3711C8400422B092D99AC17DF5CD6F49
:104110003E8A3914A572D4286756D489D2B3E9638C
:104120005DD2DA0349A9DBCD473CE3EBBFF4755719
:10413000ECEE9BF29BBE5634CCA2F2FF0308F89142
:1041400055003F091BE09B4803FCE06E80EFDC1D3F
:10415000F0831B02A72855A11A6080A74C475C4D2D
:10416000A9A6AED9E94AABAAF0E42D23CB762B83DE
:1041700037CF6CA4C95FB8EBEA91C43C916A8B530A
:104180001C4AA4A9D742E014A52A54038000CE8576
:10419000082027F7FF070A88294C0225AB4EB4CC2C
:1041A0006B9E224789F2AA7CEA1ADC3AEDCEAD6F0B
:1041B00077873BCF7D9CD5BA75EAE27EB5AB058D9E
:1041C000965CE2CE3E3993CA0D03BE37D580053CDE
:1041D00060010D00029EE7B08000A65E47401D4BC7
:1041E000FF0F0118A9CC0206284EA9143925694BE6
:1041F000BA5DAEAA84155AF5BEAB59CF61CE7D6BC0
:104200005B094976EEB51EE5692E44D39AE6277C14
:104210004D09A547DCF8B9AF7B62B770E6BE1A540A
:104220004CB8DDFF0302782D550212B080015E49C3
:104230005D4935AE1AD6F69425055B4AD755943CB0
:10424000282DFE7611CAEA06253529024528771160
:10425000D908284E151C501CD3EA6A1449F74D7B27
:104260001967534565B1A73E0814A1DC4564038076
:1042700000965653C01FAD0278AE0601CBB7FF3F84
:1042800008E8589401DF3033E07B6503FC12EA80D4
:104290005F8B1DF07BA8035E535640A11CAEF12C32
:1042A000A252DDA43A2BCC718937EA2C335DA1CD23
:1042B0002A92EC56E736230F7E4B4CD68C3CDA69BB
:1042C000355EDDEA68B755A96F1982BD1495BE61E8
:1042D000F176C385FB8825E829637387C0294A5591
:1042E000A8060008A094620C20A0A4200494E2F682
:1042F000FF0418CE4D021AD0800446915557076D21
:10430000D9CDAE4F555D5987AEB9D56D5BDB7D9389
:10431000B6EDEEE35A6B6AF491D5736B67F547BC63
:10432000D4A79CA534E4D0A6F0E4AAB82DABC39BD7
:1043300062C2AC74F69FFB720BEC92CDEECF436978
:104340004C5BFF3F0AB89CC400BF681AE03FF10015
:10435000FC24E9809F2C0D708447A93AD211976CF8
:10436000A3AAC4D68CB3AC32B31A57E9B2EACC7B59
:10437000C2B8EBAA93E871936EAB49AA3B9DFBB51B
:1043800036A8AD50E9DB8660A75CB44B1A5DAD542E
:10439000F65DE9363D4A281787CBB40E63DDED6E36
:1043A000533A5DB8B37B6C5A77E53EEEB3ADC5D5F5
:1043B000F6FC3F0E18A234004B0E2B205BB751A425
:1043C000945AAEA556994B6BBACC5D758E63D632B6
:1043D0006735398F5AEB9C3516BF262D4BD658EDD5
:1043E000398DAE5947D31BDCD2669C5DB6C9E8EA6D
:1043F00076379F626D8BCBD342888C2D2A6F8B6A68
:104400001E36A57CD5B1BB78E2F2564B6EEA4ECA99
:104410005B3D87A839096F75E2A66AF7FF0104F8CA
:10442000A5830312B0800722B0C2EE8D457DC9CAB4
:10443000672942F5353BDFF928660D40CFD7B31C1D
:10444000CDAC0614B5680E7DEE4BDFD2395B02446D
:10445000BDCE57BEF29DEE550AC1734D7EF2F3FFFD
:10446000664EA87A8DEDC4B5CD89D4BCA2DBD12728
:10447000BE334CD94F9B4D578A76BEF5A9AA2E4F15
:10448000D5CDB7D9435B87134C0DA775AB7B3EE306
:10449000196F7FA7A7F9D0305B1D9E9A3444BCB634
:1044A0007DFE1F654AEA3A5CB2CE6E57A748E6D257
:1044B0005DBBEC6217BBDE7D9FDA5C5C7AAAB56EF1
:1044C000CBD00EAD6EAFEEF98867BCDC3DAC60B80A
:1044D00045F3B7BFC3DDA2BBABCD898F7FFE1F0203
:1044E000F849CC00BF873BE0B76003FC9AAA803F45
:1044F000921130299A0286345F651369E2DA6535D4
:10450000598F495997D5657D29A5DE5697F5858E32
:10451000E45D6D0E2339DC79D4A5357572EF5195C4
:10452000E938E6B94B5D1A266B3B46E014A52A54E0
:1045300003400143BA31607335044E51AA4235FE3F
:104540001F0868210D030428CE9203234ACAA61C23
:10455000DAADB470ED1964B7D39145513589EA6687
:10456000DEEAE0ABD3294F1FFA52F690523B257F8B
:10457000DDCB9D72728C79CB6FFAD2109EB42CE198
:104580004F25703ADCBA2F6FC175CBF2FF0AA8BA7B
:10459000B814DD9C9298EB5554DDA6619D57DB78ED
:1045A000BBA66E5E6DE36E99DCB8745589AF70F48E
:1045B000D46745DD6C7655194446B13932C0B0C573
:1045C0000E18B65301C198942A144B09C9B2AA68AF
:1045D0002A3DD8FB2A93987663EFA7CC6C3A8DB32B
:1045E000AE2AB1ED64C932EA82674A286B6B33A9FF
:1045F0006994ACBD2D43D4DD019A2F4C59C938AA1A
:10460000DFFF076EADCC349C97E823ED5DA4BBF1D2
:1046100096D9EEFAD44575A6C9E65BDFE60E67AE1D
:104620007CD343FBEC7D9EFDFE7F08D8849901CFAF
:10463000B832E0A71405FC566A8100FC96EA805F58
:10464000CA563E79AAAAB75E45D3A96AF96415DDB0
:10465000B499C69A55D45062D6B54BD6784B58CD3E
:1046600044E014A52A5403001430853A039EAFF8A1
:104670007F00B09CEC3AB942F271739C946939C7DF
:10468000C9B94336651F3797765EB373BC12A6A8C7
:10469000D3F6F1522F93553B2748334557148F30AB
:1046A000E5315CA1D3C26CDA205D4E088B1F463326
:1046B000382E2EF982D3201120460302281702003B
:1046C00000000000F000D0CC2C58A62BF0319B222B
:1046D000EAEA51C76C8AB0AB471DB34AC2EAAA7C6A
:1046E000EC660833A7CCB19B21CC9C22CBAE8AB020
:1046F000AA8B0C270BD4CD0A33DC2251BB364C716C
:104700000367FF0EB3C113D2EA53C51A0FEBD815D6
:1047100013CB7CA46D37C32EF1B5A49A2E3B0000B9
:1047200000000000F0000420332505AA34695495E8
:1047300016A832A45E514B205BA366452E81684DBE
:1047400092553905AC2D73649410D2D5AC51515C9F
:10475000C29F624CD876099B85EA994464708FB0F9
:104760007B6C91825E6CE189592A93BB8AD82125A2
:10477000F3E6AE16190000000000001E00104C8F7A
:10478000B3AFD072733350BF4547C36B40644E6DB7
:104790000FAF42967D953CFC82597F59720B326275
:1047A000FB25C923CC48FC9725B738018D5F96546B
:1047B0009200A3BEC9544A03D2FCD48826252CEB10
:1047C000C223899CF1ACF128C90A4738276211003D
:1047D00000000000003C0030EC64C53957F2715213
:1047E00064F15C3BC74DCAD465231F2F4B33970937
:1047F0007DBC64D425D6F2F19355B1D8D02B484E68
:1048000055E24C8F301A358DB33C92684C3DCE74D6
:104810004BBC53CB5AD121E5DE32BBC1A80C258B52
:10482000A902CD5261C57D47340000000000003C64
:104830006D17AA7AC24C8DD5739DAD0835562B7471
:104840003AD3E458A4B2C92C516749DCCCAB2A9FB7
:10485000AD6837F1AA75F6AA2C35A3D239B288D241
:10486000CC90E74C3C2ACC639EBF0B7577AD75FEB0
:104870002ADCD47C3618A072310000786BAF9245E8
:10488000E65A8D234AF6DC6A3876AFD46BDBE1DA80
:1048900093269DEE96676F01C5BA579EBD5962DBA0
:1048A0005974CE2E58786EE1BA3A65D1B98A0A00A9
:1048B000EE1A1E8DDC797283931A60E954036C65DD
:1048C0006A8029420C3045EA298B30B3E8C867ADCD
:1048D000D64CB36A9FA37A0DADAA75EAA6B9622237
:1048E000E2A9BB36A70A2BA34EDC22A642ABDA0311
:1048F000358B8C4CEA8658542D0E903A11B674B70D
:104900000DF00DBDB143C56A076069D7004C931C1B
:10491000802D9303B07468028E3639CD92C29C33D9
:10492000F94C1DB3C76CE433572416BB91CF363115
:10493000C6CC543E7B8354BD13E95C93A1656FEDF7
:10494000D39DAA8A304B4E77EA4400C65EDDCE3B4B
:10495000C31C6B7533FD8C69ECD6EDB095625512B6
:10496000BA435788C74EE80E53A91A37E1C74DB965
:1049700059DC441DDF156A49000040001588C0035A
:1049800089BCA9D39D132B607257050CAAA2802164
:104990009C0DB0A49903A6084D00316DA72D369546
:1049A000DD1A9FA1C452744F72E6BC8D24CCC95944
:1049B000F3700AF6D8674FC9D935629F3D8954779D
:1049C00073738EC4C3B52DCE393A56E7AC38E7ECD5
:1049D00054D426639FAB12B69A8E5C36CDB6BB44D8
:1049E000B4DA389FCA324A6CCB9055CC9CB0E646BC
:1049F0001662B10CA97923DD442D97E6B7728FB00A
:104A0000D49A77C74324716BDE9870D1DAA5B9B315
:104A100055551B3F275FC1443CE39CA15A53CD8CA5
:104A20007586E63C82D5D159ABAF3055CB676BAEBE
:104A30002DC4CD9CBD1977B1B494D0C2C5295312F1
:104A4000430B50B5F04408ED4444446C1300F00CA3
:104A500080464E1B61EE510FD96D97B93A1D7873A0
:104A6000571929B7A143CF849AA59537BB19A176C9
:104A700046DEEC9799596E79755FA626FA01059086
:104A80003CD501589FAE7A8018674DB416C7BFC594
:104A9000A4C958B8FF10972A6BE3F1934D639FDDCB
:104AA000DA2FD288728E10BE5933CA39A2DD51AEC8
:104AB0004AE7C9EE4BB9269DAE981BC7ACB4BAAA5B
:104AC0007A0DB2E4E8B2BF66E940A5CBFE5B240BE9
:104AD000C3030030C64549253CCE198E541753DB1D
:104AE000674C3852B31B9DD1E84EBDAE74262F2AB9
:104AF0007426D659BC4A979D8A6B75B2D2B226AC41
:104B0000D5F1EA71ABD95627B3326AE203A76A3A04
:104B100032C45D9F2AE736F19675AA5CCB4CCBD6A2
:104B2000A9F274314B47A74A4DD82B649F3A6B7357
:104B3000B548B5EA9CDCC0BD363CA72B5234A66A0A
:104B40009E290AB3E98C74A64C5D7D3AD25A1A3775
:104B5000D6E83AAB9FB604C963AF6DD916448BB3A0
:104B6000A6659C89A3F6698632268FDAA7E85644A3
:104B7000B2969C742A15E95C7D92C63862B3D1491D
:104B80002A57D7F4CC27EDC4CB58DDAEA2A31A2602
:104B900069B2AA0E628CA5E9AA33AA09E174A78DAD
:104BA000B4D748BB9E36D21943DDB2DA827C47B017
:104BB000DB6A13CE1DC5ECAD7572D7995795C38BC3
:104BC0001DA2581516AD6F4173163CA74D69CAB5A5
:104BD000E69CBE8AEE35AE73FA26BAC778C9E9AA52
:104BE000EA1E91BA67A8BAA6C5EA9C21876EE78A31
:104BF00072A6ECB682B24E9B8A9D112A51F06B2DA3
:104C00008AD9A7369EB11B21CDEE7BA66E99B8BA84
:104C1000DF99BA63E6AA3E676A96C43A1B02C003EC
:104C20002397E1CA5196AE5CA61E056F7A0A197ADF
:104C30001235E92AA49B69A2A4ABD46AFA1493AEF4
:104C4000CA8AEE0B70326AC7AB2FC8093C273F8671
:104C500059245F9D6220D2ACB9748A8151ABFBD6D6
:104C6000C92721F59ADB279F94C572AE9C7C096603
:104C7000F6B9738A49D1AA77E4AA27458BDA426943
:104C8000CC406AD32DC303A7695223CA7B9DA64992
:104C9000C95ACB7CEAA6C523B4F5699A3213932E80
:104CA000A7AB2A8CD45A0300003CE43811241FBE61
:104CB000CFEFD8E0DEBFCDBF24E0ACE2B3E001C06F
:104CC0001D92AC35B207E1F713E0A0E0B1E0E4E7F4
:104CD000FBE702C005900D92AC32B107D9F716E29E
:104CE000C6E5D6E204C02197FE010E943639C535DB
:104CF000D107C9F70E94CA330C94B83D0C94000048
:104D0000CF92DF92EF92FF920F931F93CF93DF9397
:104D10006C017A018B01C0E0D0E0CE15DF0589F08F
:104D2000D8016D918D01D601ED91FC910190F0813A
:104D3000E02DC6010995892B11F47E0102C0219650
:104D4000ECCFC701DF91CF911F910F91FF90EF90B2
:104D5000DF90CF900895FC01918D828D981761F0BE
:104D6000828DDF01A80FB11D5D968C91928D9F5FA2
:104D70009F73928F90E008958FEF9FEF0895FC014D
:104D8000918D828D981731F0828DE80FF11D858D00
:104D900090E008958FEF9FEF0895FC01918D228D93
:104DA000892F90E0805C9F4F821B91098F73992718
:104DB000089584EB93E00E94CD2621E0892B09F42D
:104DC00020E0822F0895FC01848DDF01A80FB11D22
:104DD000A35ABF4F2C91848D90E001968F73992731
:104DE000848FA689B7892C93A089B1898C9180641E
:104DF0008C93938D848D981306C00288F389E02DDF
:104E000080818F7D80830895EF92FF920F931F938F
:104E1000CF93DF93EC0181E0888F9B8D8C8D98136D
:104E200005C0E889F989808185FD24C0F62E0B8DA7
:104E300010E00F5F1F4F0F731127E02E8C8DE812CB
:104E40000CC00FB607FCFACFE889F989808185FF8D
:104E5000F5CFCE010E94E326F1CF8B8DFE01E80F46
:104E6000F11DE35AFF4FF0820B8FEA89FB898081A5
:104E7000806207C0EE89FF896083E889F9898081B3
:104E80008064808381E090E0DF91CF911F910F914A
:104E9000FF90EF900895CF93DF93EC01888D8823E6
:104EA000C9F0EA89FB89808185FD05C0A889B98997
:104EB0008C9186FD0FC00FB607FCF5CF808185FF72
:104EC000F2CFA889B9898C9185FFEDCFCE010E94E0
:104ED000E326E7CFDF91CF91089580E090E0892B22
:104EE00029F00E94D92681110C9400000895833086
:104EF00081F028F4813099F08230A1F00895873054
:104F0000A9F08830B9F08430D1F4809180008F7D91
:104F100003C0809180008F7780938000089584B5CE
:104F20008F7702C084B58F7D84BD08958091B000D5
:104F30008F7703C08091B0008F7D8093B00008957B
:104F40001F93CF93DF93282F30E0F901EF58F94DED
:104F50008491F901ED52F14DD491F901E154F14DF3
:104F6000C491CC23C9F0162F81110E947727EC2F12
:104F7000F0E0EE0FFF1FE959F94DA591B4918FB7FD
:104F8000F894111105C09C91ED2FE095E92302C022
:104F9000EC91ED2BEC938FBFDF91CF911F91089592
:104FA0003FB7F8948091590390915A03A0915B0305
:104FB000B0915C0326B5A89B05C02F3F19F0019660
:104FC000A11DB11D3FBFBA2FA92F982F8827820F8F
:104FD000911DA11DB11DBC01CD0142E0660F771FDF
:104FE000881F991F4A95D1F708950E94F43C1F929B
:104FF0000F920FB60F9211242F933F934F935F930D
:105000006F937F938F939F93AF93BF93EF93FF9390
:1050100084EB93E00E94E326FF91EF91BF91AF9163
:105020009F918F917F916F915F914F913F912F91C0
:105030000F900FBE0F901F9018951F920F920FB6F2
:105040000F9211242F938F939F93EF93FF93E091EF
:10505000C403F091C5038081E091CA03F091CB03B2
:1050600082FD12C090818091CD038F5F8F7320915C
:10507000CE03821751F0E091CD03F0E0EC54FC4FE9
:10508000958F8093CD0301C08081FF91EF919F9117
:105090008F912F910F900FBE0F901F901895CF9367
:1050A000DF93282F30E0F901EF58F94D8491F90191
:1050B000ED52F14DD491F901E154F14DC491CC235D
:1050C00091F081110E947727EC2FF0E0EE0FFF1F87
:1050D000EF55F14DA591B491EC91ED2381E090E075
:1050E00021F480E002C080E090E0DF91CF9108954C
:1050F000CF9386E00E944F28892BA1F087E00E9481
:105100004F28892B31F080914203909143030197FE
:1051100005C080914203909143030196909343030D
:1051200080934203809142039091430397FD0BC00B
:105130008091420390914303839744F4809142030A
:105140009091430305C080E090E002C082E290E0CD
:1051500090934303809342038091420390914303D1
:1051600097FD019695958795809356048A3010F0A7
:1051700061E001C060E08DE00E94A02780915604AC
:105180006AE00E941639C92F692F66956695669563
:105190008CE00E94A027C2FB662760F98BE00E948A
:1051A000A027C1FB662760F98AE00E94A0276C2F28
:1051B000617089E0CF910C94A027CF93DF9390E0AA
:1051C000FC01ED52F14D2491FC01E154F14D84912B
:1051D000882361F190E0880F991FFC01E35AF94D93
:1051E000C591D491FC01E959F94DA591B491611192
:1051F00009C09FB7F8948881209582238883EC9119
:105200002E230BC0623061F49FB7F8943881822F4F
:10521000809583238883EC912E2B2C939FBF06C00F
:105220008FB7F894E8812E2B28838FBFDF91CF9121
:1052300008958E3008F08E508770806480937C00D3
:1052400080917A00806480937A0080917A0086FD54
:10525000FCCF809178002091790090E0922B089506
:105260008F929F92AF92BF92CF92DF92EF92FF9276
:105270006B017C010E94D0274B015C01C114D10459
:10528000E104F104F1F00E94D027DC01CB01881980
:105290009909AA09BB09883E9340A105B10570F39D
:1052A00021E0C21AD108E108F10888EE880E83E0F7
:1052B000981EA11CB11CC114D104E104F10419F71A
:1052C000DDCFFF90EF90DF90CF90BF90AF909F9099
:1052D0008F9008951F920F920FB60F9211242F9363
:1052E0003F938F939F93AF93BF938091550390917A
:1052F0005603A0915703B09158033091540323E013
:10530000230F2D3720F40196A11DB11D05C026E8FD
:10531000230F0296A11DB11D2093540380935503C2
:1053200090935603A0935703B09358038091590369
:1053300090915A03A0915B03B0915C030196A11D6B
:10534000B11D8093590390935A03A0935B03B093CC
:105350005C03BF91AF919F918F913F912F910F90DF
:105360000FBE0F901F9018956093500370935103D8
:105370008093520390935303DC01CB01845D9E4FD5
:10538000AF4FBF4F80934C0390934D03A0934E03B8
:10539000B0934F0382E090E090934B0380934A03D5
:1053A0002FB7F8948091550390915603A09157031D
:1053B000B09158032FBF8093460390934703A09367
:1053C0004803B093490308950F931F938FB7F89440
:1053D00000915503109156032091570330915803C3
:1053E0008FBF4091460350914703609148037091ED
:1053F0004903041B150B260B370B8091500390912A
:105400005103A0915203B0915303083E134021056C
:105410003105C0F00196A11DB11D809350039093FA
:105420005103A0935203B093530348515C4F6F4F05
:105430007F4F409346035093470360934803709314
:105440004903C4CF40914C0350914D0360914E03EA
:1054500070914F0384179507A607B70788F1E0916D
:105460004403F0914503309759F109956115710591
:105470008105910519F00E94B42922C08091500342
:1054800090915103A0915203B0915303845D9E4FBC
:10549000AF4FBF4F80934C0390934D03A0934E03A7
:1054A000B0934F0381E090E020914A0330914B0389
:1054B000232B11F480E090E090934B0380934A03F8
:1054C0006091500370915103809152039091530366
:1054D0001F910F91089501978533910508F09FC0A2
:1054E0008C5C9F4FFC010C94363985E79AE395C09C
:1054F00081ED95E292C085E495E28FC087ED94E25C
:105500008CC08AE694E289C086EE93E286C082E689
:1055100093E283C084EE92E280C08DE895E47DC082
:105520008AE692E27AC089E092E277C089EA91E263
:1055300074C08FE491E271C08FE399E36EC085EF90
:1055400090E26BC08EE890E268C08FE090E265C0A8
:1055500085E69FE162C088EF9EE15FC082EA9DE13F
:105560005CC08EE19DE159C083EC9CE156C081E8AE
:105570009CE153C086E29CE150C083E99BE14DC0B1
:105580008CEC9AE14AC08EE49AE147C08AE999E13D
:1055900044C08AE09EE141C083E099E13EC08EE5CF
:1055A00098E13BC08BEC97E138C089E797E135C0C3
:1055B0008EE297E132C083ED96E12FC089E896E153
:1055C0002CC08DE196E129C080EB95E126C08FE4E7
:1055D00095E123C088E994E120C08AEE93E11DC0E3
:1055E0008BE493E11AC08CE093E117C081EA92E169
:1055F00014C08AE392E111C08FED98E30EC08FEDE5
:1056000091E10BC08FE29AE308C085EC99E305C0F5
:1056100089E99EE302C08EE19BE30C94D8300895A3
:1056200001978A31910508F054C087599F4FFC01BA
:105630000C9436398BE791E14AC083E291E147C08F
:1056400081EC90E144C08EE690E141C08CE290E1B3
:105650003EC087E99FE03BC08FE59FE038C089EE00
:105660009EE035C089E89EE032C083E29EE02FC014
:1056700086ED9DE02CC083E99DE029C081E59DE099
:1056800026C085EB9CE023C088E59CE020C086E135
:105690009CE01DC08FEC9BE01AC08FE69BE017C01A
:1056A00089ED9AE014C082E69AE011C084EE99E098
:1056B0000EC081E799E00BC088E199E008C084EA58
:1056C00098E005C081E498E002C088EF97E00C9470
:1056D000D8300895CF92DF92EF92FF920F931F93ED
:1056E000CF93DF936B017C01F7FE0DC088EA97E052
:1056F0000E94D830F094E094D094C094C11CD11C86
:10570000E11CF11CF1CFC114D104E104F10419F43E
:105710008BE597E0D7C088EEC81683E0D806E10491
:10572000F10414F1C701B60128EE33E040E050E087
:105730000E94553D8B01D82FC92FB901330F880B1B
:10574000990B0E946A2B82EE96E00E94D830680185
:10575000ED2EFC2ED701C6010197A109B1098336B0
:105760009105A105B10510F184E6C816D104E10444
:10577000F10404F1C701B60124E630E040E050E056
:105780000E94553D8B01D82FC92FCA01B9010E9433
:105790006A2B84E396E00E94D8306801ED2EFC2E3F
:1057A000C114D104E104F10409F496C08BE896E039
:1057B0000E94D83084E1C816D104E104F104E4F178
:1057C000C701B6012AE030E040E050E00E94553DBC
:1057D000C901330FAA0BBB0BFC013397E730F1056E
:1057E00020F4ED57FF4F0C94363988EE95E018C041
:1057F00080EB95E011C081E495E40EC080E595E072
:105800000BC08EE195E008C084ED94E005C081EA0C
:1058100094E002C089E494E00E94D83086E795E0E5
:105820000E94D830C701B6012AE030E040E050E0E5
:105830000E94553D6B017C01F6013197E331F10582
:1058400008F04AC0E657FF4F0C94363980E694E4DE
:1058500039C082E194E036C086EC93E033C081E445
:1058600095E430C083E793E02DC08EE195E02AC037
:1058700084ED94E027C081EA94E024C089E494E0B8
:1058800021C08DE393E01EC085ED92E01BC08CE843
:1058900092E018C080EB95E011C081E495E40EC061
:1058A00080E595E00BC08EE195E008C084ED94E0C2
:1058B00005C081EA94E002C089E494E00E94D830F7
:1058C00086E592E0DF91CF911F910F91FF90EF90CD
:1058D000DF90CF900C94D830DF91CF911F910F9132
:1058E000FF90EF90DF90CF9008951F920F920FB628
:1058F0000F9211242F933F934F935F936F937F9356
:105900008F939F93AF93BF93CF93EF93FF9329B15F
:10591000C091610390918F0380918C03322F309559
:1059200083239223892B90916D00C227C923C8231A
:1059300020936103CC23C1F1C0FF05C0E091620355
:10594000F09163030995C1FF05C0E0916403F091F4
:1059500065030995C2FF05C0E0916603F0916703F6
:105960000995C3FF05C0E0916803F09169030995AB
:10597000C4FF05C0E0916A03F0916B030995C5FF70
:1059800005C0E0916C03F0916D030995C6FF05C059
:10599000E0916E03F0916F030995C7FF05C0E09198
:1059A0007003F09171030995FF91EF91CF91BF9131
:1059B000AF919F918F917F916F915F914F913F91A7
:1059C0002F910F900FBE0F901F9018951F920F925E
:1059D0000FB60F9211242F933F934F935F936F93C2
:1059E0007F938F939F93AF93BF93CF93EF93FF9347
:1059F00026B1C09172039091900380918D03322F54
:105A0000309583239223892B90916C00C227C92360
:105A1000C82320937203CC2351F1C0FF05C0E0914D
:105A20007303F09174030995C1FF05C0E0917503FC
:105A3000F09176030995C2FF05C0E0917703F091DC
:105A400078030995C3FF05C0E0917903F0917A03CB
:105A50000995C4FF05C0E0917B03F0917C03099593
:105A6000C5FF05C0E0917D03F0917E030995FF918C
:105A7000EF91CF91BF91AF919F918F917F916F9156
:105A80005F914F913F912F910F900FBE0F901F90FC
:105A900018951F920F920FB60F9211242F933F93D8
:105AA0004F935F936F937F938F939F93AF93BF9326
:105AB000CF93EF93FF9323B1C0917F039091910314
:105AC00080918E03322F309583239223892B9091DE
:105AD0006B00C227C923C82320937F03CC2351F135
:105AE000C0FF05C0E0918003F09181030995C1FFDB
:105AF00005C0E0918203F09183030995C2FF05C0C0
:105B0000E0918403F09185030995C3FF05C0E091FE
:105B10008603F09187030995C4FF05C0E0918803CF
:105B2000F09189030995C5FF05C0E0918A03F091C2
:105B30008B030995FF91EF91CF91BF91AF919F9109
:105B40008F917F916F915F914F913F912F910F9026
:105B50000FBE0F901F9018951F920F920FB60F92C5
:105B600011242F933F934F935F936F937F938F9362
:105B70009F93AF93BF93EF93FF93E0915F03F091F7
:105B800060030995FF91EF91BF91AF919F918F9124
:105B90007F916F915F914F913F912F910F900FBE29
:105BA0000F901F9018951F920F920FB60F9211240D
:105BB0002F933F934F935F936F937F938F939F9315
:105BC000AF93BF93EF93FF93E0915D03F0915E037A
:105BD0000995FF91EF91BF91AF919F918F917F9127
:105BE0006F915F914F913F912F910F900FBE0F904A
:105BF0001F9018951F920F920FB60F9211242F929B
:105C00003F924F925F926F927F928F929F92AF924C
:105C1000BF92CF92DF92EF92FF920F931F932F9339
:105C20003F934F935F936F937F938F939F93AF9324
:105C3000BF93EF93FF93CF93DF93CDB7DEB7A497D6
:105C4000DEBFCDBF809141038093B40078949091E2
:105C5000A603992309F180914003891720F48F5FEF
:105C60008093400302C010924003E0914003E93268
:105C700088F5F0E0EA5FFE4FA0812091B2033091F9
:105C8000B3030A2E000CBB0B0E944439BB27A92F7B
:105C9000982F872FBC0120C0209100013091010175
:105CA000C90196958795A9014170552720FF02C02B
:105CB00040E058EB842795279093010180930001E1
:105CC0006091B2037091B30380FD06C07195619538
:105CD000710902C060E070E0E091A8034E2FEE0F62
:105CE000550B5AA349A360903C0370903D0340912B
:105CF000A70320913E0330913F034203C001439F1D
:105D0000900D1124880F892F881F990B681B790B20
:105D1000E9A1FAA1E69DC001E79D900DF69D900DC9
:105D20001124880F892F881F990B4B01881A990A13
:105D30004090A903042C000C550840913A0350915F
:105D40003B035A834983449EC001459E900D549E57
:105D5000900D1124880F892F881F990B1401281A80
:105D6000390A8091A503E82F880FFF0BFC83EB8392
:105D700040913803509139035E834D83E49FC00105
:105D8000E59F900DF49F900D1124880F892F881F97
:105D9000990BF101E81BF90BF887EF838091AA03B7
:105DA000482F880F550B5A874987E0913603F091A9
:105DB0003703FC87EB874E9FC0014F9F900D5E9F7E
:105DC000900D1124880F892F881F990B4F815885BA
:105DD000481B590B5E874D878091AB03E82F880FD6
:105DE000FF0BF88BEF8740913403509135035A8BAA
:105DF000498BE49FC001E59F900DF49F900D112405
:105E0000880F892F881F990BED85FE85E81BF90BFC
:105E1000FC8BEB8B8091AC03482F880F550B5E8B6E
:105E20004D8BE0913203F0913303F88FEF8B4E9F4F
:105E3000C0014F9F900D5E9F900D1124880F892FF8
:105E4000881F990B4B895C89481B590B5A8F498FC6
:105E50008091AD03E82F880FFF0BFC8FEB8F4091F3
:105E60003003509131035E8F4D8FE49FC001E59F59
:105E7000900DF49F900D1124880F892F881F990B86
:105E8000E98DFA8DE81BF90BF8A3EF8FA090AE0314
:105E9000B090AF03E0902E03F0902F039501D7014F
:105EA0000E943C39DC01CB014FE0B595A795979551
:105EB00087954A95D1F76F01C81AD90A0091B003A6
:105EC0001091B10340912C0350912D035CA34BA37F
:105ED0009801DA010E943C39DC01CB015FE0B59505
:105EE000A795979587955A95D1F7A601481B590B09
:105EF000411562E056073CF441157EEF57072CF43C
:105F000040E05EEF02C04FEF51E0E9A1FAA1E89D49
:105F1000C001E99D900DF89D900D1124880F892FE7
:105F2000881F990B860D971D90933F0380933E0326
:105F3000429CC001439C900D529C900D1124880FEF
:105F4000892F881F990BE981FA818E0F9F1F9093EB
:105F50003D0380933C03EB81FC812F813885E29FD8
:105F6000C001E39F900DF29F900D1124880F892F9F
:105F7000881F990BED81FE818E0F9F1F90933B032D
:105F800080933A03E985FA852D853E85E29FC0011D
:105F9000E39F900DF29F900D1124880F892F881F89
:105FA000990BEB85FC858E0F9F1F9093390380938F
:105FB0003803EF85F8892B893C89E29FC001E39F74
:105FC000900DF29F900D1124880F892F881F990B37
:105FD000E989FA898E0F9F1F9093370380933603C8
:105FE000ED89FE89298D3A8DE29FC001E39F900DD6
:105FF000F29F900D1124880F892F881F990BEF892C
:10600000F88D8E0F9F1F9093350380933403EB8D93
:10601000FC8D2F8D38A1E29FC001E39F900DF29F70
:10602000900D1124880F892F881F990BED8DFE8DFF
:106030008E0F9F1F90933303809332039501D601F7
:106040000E943C39DC01CB012FE0B595A7959795CF
:1060500087952A95D1F7B701680F791F709331039F
:10606000609330039801DA010E943C39DC01CB01D6
:106070003FE0B595A795979587953A95D1F7EBA110
:10608000FCA18E0F9F1F90932F0380932E0350939C
:106090002D0340932C0355954795559547954058AA
:1060A00040934103A4960FB6F894DEBF0FBECDBF58
:1060B000DF91CF91FF91EF91BF91AF919F918F9120
:1060C0007F916F915F914F913F912F911F910F9110
:1060D000FF90EF90DF90CF90BF90AF909F908F9008
:1060E0007F906F905F904F903F902F900F900FBEDA
:1060F0000F901F901895CF93DF93A0915104B0910A
:106100005204FD0144914295942F9373F4E09F9FB4
:10611000900111244C7C46954695242B922F957521
:10612000990F2A7A2695292B30E0322F2227709159
:106130005304C82FD0E0AE01470F511D493051051F
:10614000B4F0FD0131964491642F6295962F9373BC
:10615000E4E09E9FA00111246C7C66956695462B19
:10616000942F9575990F4A7A4695492B242B072E23
:1061700002C0220F331F0A94E2F740E150E04C1BAB
:106180005D0B02C0369527954A95E2F7780F783077
:1061900018F47093530408C0785070935304119608
:1061A000B0935204A0935104822FDF91CF910895B0
:1061B0004F925F926F927F928F929F92AF92BF9217
:1061C000CF92DF92EF92FF921F93CF93DF93EC0178
:1061D00080915704811120C061E083E00E94DD2896
:1061E00083E28093B00091E09093B1001092700030
:1061F0001092800089E080938100109285001092B7
:10620000840020ED37E0309389002093880082E0FD
:1062100080936F0090935704D0935204C09351041D
:1062200010925304CC24CA9423E0D22EE12CF12CFA
:10623000412C34E2532E34EF632E712C44ED842E26
:1062400043E0942EA12CB12C8091540490915504DC
:10625000019711F581E00E941929BC01990F880B63
:10626000990B0E94093A9B01AC0168E77FE680E840
:106270009FE30E94023B20E639EE44E853E40E948B
:10628000953A0E94D13960935804709359048093D1
:106290005A0490935B041AC081E00E94192928E2F5
:1062A00033E2DC010E944439A70196010E94553D6A
:1062B000DA01C90188519C4FAF4FBF4F80935804FA
:1062C00090935904A0935A04B0935B04209158040E
:1062D0003091590440915A0450915B04C301B201BA
:1062E0000E94553D309389002093880084E00E94ED
:1062F0007B30C82F8091540490915504029739F453
:10630000C11126C01092B3031092B20328C182E0DB
:106310000E944F28892BA1F71092B3031092B20369
:106320001092B1031092B0031092AF031092AE031B
:106330001092AD031092AC031092AB031092AA031B
:106340001092A9031092A8031092A703CFE007C1EF
:10635000CF3011F3EC2FF0E0E45FFC4F808190E050
:106360009093B3038093B20381E00E947B30182F97
:1063700086E00E947B30E82FF0E0E453FD4FD081AF
:10638000D093A60380915404909155040197D9F5B8
:106390001123D9F1DD2309F4E2C083E00E94192919
:1063A0009C01A2ECBFEF0E943C39A70196010E941C
:1063B000553DDA01C901CF96A11DB11D8093A603F9
:1063C00083E00E941929892B11F41092A603809171
:1063D000A603811115C082E00E9419299C01A1EF3A
:1063E000BFEF0E943C39A70196010E94553DDA019A
:1063F000C9010F96A11DB11D9093B3038093B20301
:106400004A99CBCFACC01111AAC085E00E947B3065
:10641000E82FF0E0EE0FFF1FE457FD4F80819181E0
:106420009093B1038093B00385E00E947B30E82F06
:10643000F0E0EE0FFF1FE45BFD4F808191819093B0
:10644000AF038093AE0384E00E947B30E82FF0E03E
:10645000E45CFD4F80818093AD0384E00E947B303B
:10646000E82FF0E0E45DFD4F80818093AC03DD23F5
:1064700009F475C084E00E947B30E82FF0E0E45E10
:10648000FD4F80818093AB0384E00E947B30E82F36
:10649000F0E0E45FFD4F80818093AA0384E00E94D6
:1064A0007B30E82FF0E0E450FE4F80818093A5031D
:1064B00083E00E947B30E82FF0E0EC50FE4F8081BB
:1064C0008093A90383E00E947B30E82FF0E0E45141
:1064D000FE4F80818093A80383E00E947B30E82FE9
:1064E000F0E0EC51FE4F80818093A70384E00E948E
:1064F0004F28892BA1F583E00E941929092E000C51
:10650000AA0BBB0B9C01AD01245131094109510972
:10651000AEE6B0E00E94743DA50194010E94553D95
:106520002093AB0383E00E941929092E000CAA0BCB
:10653000BB0B9C01AD012451310941095109AAE667
:10654000BFEF0E94823DA50194010E94553DDA01F2
:10655000C9018A569F4FAF4FBF4F8093A70382E078
:106560000E9419292091540430915504213031059D
:1065700089F09C01ACE9BFEF0E943C39A70196016C
:106580000E94553DDA01C9018C599F4FAF4FBF4F53
:10659000BC0102C060E070E0072E000C880B990B74
:1065A0000E943029CF3009F04FCE80915404909151
:1065B0005504029729F082E00E944F28892BD9F3D5
:1065C000DF91CF911F91FF90EF90DF90CF90BF9020
:1065D000AF909F908F907F906F905F904F900895B5
:1065E0004F925F926F927F928F929F92CF92DF92A3
:1065F000EF92FF920F931F93CF93DF932CE3C22E62
:10660000D12CE12CF12CA70196010E94873D6093CB
:106610009E03CA01B901A70196010E94873D6093BC
:106620009F03CA01B90128E130E040E050E00E9438
:10663000873D29013A016093A003CA01B9016C5F4B
:106640007F4F8F4F9F4F27E030E040E050E00E94A7
:10665000873D6F5F6093A103C12CD12C760120E0B0
:1066600004E610E030E9832E99249394E22FF0E0C1
:10667000EE54F84FEF01C370DD27209789F4CF0166
:10668000B8010E942239892B31F4CF01B4010E9454
:106690002239892B29F48EE691E0A0E0B0E004C015
:1066A0008DE691E0A0E0B0E0C80ED91EEA1EFB1E08
:1066B000D701C601AA27BB27481659066A067B06DA
:1066C00010F02F5FD3CF2093A403209799F4CF012C
:1066D00064E670E00E942239892B39F4CF0160E929
:1066E00071E00E942239892B29F48EE691E0A0E026
:1066F000B0E004C08DE691E0A0E0B0E0C81AD90A8D
:10670000EA0AFB0A930182010C191D092E093F09AF
:10671000CF0164E670E00E9422397C01CF0160E97C
:1067200071E00E942239E8EDF1E0A0E0A13041F4EF
:10673000209751F4E114F10429F4009729F402C0E0
:10674000408103C04DE101C04CE150E060E070E0E9
:10675000041715072607370740F0041B150B260BF7
:10676000370BAF5F3196AC3009F7AF5FA093A3034F
:106770000F5F0093A203DF91CF911F910F91FF90C4
:10678000EF90DF90CF909F908F907F906F905F9071
:106790004F900895CF93DF9300D000D0CDB7DEB7F0
:1067A000789484B5826084BD84B5816084BD85B5EC
:1067B000826085BD85B5816085BD80916E008160F8
:1067C00080936E001092810080918100826080939E
:1067D00081008091810081608093810080918000A0
:1067E0008160809380008091B10084608093B100CB
:1067F0008091B00081608093B00080917A008460C5
:1068000080937A0080917A00826080937A008091F0
:106810007A00816080937A0080917A00806880930A
:106820007A001092C10080917A00887F80937A006C
:1068300080917A00856080937A0061E08DE00E940B
:10684000DD2861E089E00E94DD2861E08AE00E94A5
:10685000DD2861E08BE00E94DD2861E08CE00E9491
:10686000DD2862E084E00E94DD2862E085E00E948D
:10687000DD2862E088E00E94DD2860E082E00E947E
:10688000DD2862E087E00E94DD2862E086E00E9469
:10689000DD28EAEDFEE28491E6ECFEE2949192308E
:1068A00059F420919103282B2093910320918E037A
:1068B000282B20938E0319C0933059F42091900314
:1068C000282B2093900320918D03282B20938D0358
:1068D0000CC0943051F420918F03282B20938F0308
:1068E00020918C03282B20938C03E2EBFEE2A491F1
:1068F0009230D1F4B0E0AA0FBB1FA058BC4F28E7DC
:1069000038E22D933C93E5EAFEE2A591B4919C9187
:1069100090937F032BE630E0309393032093920310
:1069200090916800916037C09330D1F4B0E0AA0F25
:10693000BB1FAD58BC4F28E738E22D933C93E7EAE4
:10694000FEE2A591B4919C91909372032CE630E005
:1069500030939303209392039091680092601BC040
:106960009430D9F4B0E0AA0FBB1FAE59BC4F28E752
:1069700038E22D933C93E9EAFEE2A591B4919C9113
:10698000909361032DE630E03093930320939203BC
:1069900090916800946090936800A0919203B091E8
:1069A0009303EC918E2B8C9355EF852E53E0952E0F
:1069B000A12CB12CCC24CA9463E0D62EE12CF12C6E
:1069C00078EE472E73E0572E612C712C89B18072BE
:1069D00090E044E0959587954A95E1F790935504AA
:1069E0008093540423B120FB222420F8312C820D03
:1069F000931D9093550480935404029769F0E0919D
:106A000056048E2F90E08231910508F0DAC3FC0124
:106A1000E356FF4F0C94363982E00E944F280197CD
:106A2000D9F382E00E944F28892BD9F3E8CF80E088
:106A30000E94192929E030E0DC010E944439A301B9
:106A400092010E94553DCA01B901772788279927ED
:106A5000D6C080E00E94192929E030E0DC010E94C4
:106A60004439A70196010E94553D822F90E08A305B
:106A7000910508F0A6C3FC01E155FF4F0C9436398F
:106A800089E092E39CC383EA91E399C380E791E3B1
:106A900096C388E091E393C38BEA90E390C38DE2C1
:106AA00090E38DC38AEF9FE28AC382EA9FE287C3A5
:106AB0008BE59FE284C387EE9EE281C380E00E9463
:106AC000192929E130E0DC010E944439A70196012F
:106AD0000E94553DDA01C9010196A11DB11D092E83
:106AE000000CAA0BBB0BFC013197EA31F10508F051
:106AF00068C3E754FF4F0C94363985EF97E35FC3C3
:106B000083EC97E35CC38EE194E459C38FE897E389
:106B100056C389E597E353C38FE197E350C381EEF2
:106B200096E34DC386EA96E34AC384E696E347C3F9
:106B300081E296E344C380EE95E341C381EA95E3A5
:106B40003EC382E695E33BC382E295E338C384EF1C
:106B500094E335C38EEB94E332C38AE894E32FC306
:106B60008EE594E32CC38EE294E329C384EF93E390
:106B700026C386EB93E323C382E693E320C38CEF23
:106B800092E31DC383EC92E31AC381E892E317C337
:106B900085E492E314C380E00E94192929E130E0E2
:106BA000DC010E944439A30192010E94553DDA01A3
:106BB000C9010196A11DB11D0E94102B02C380E0E6
:106BC0000E94192924E330E0DC010E944439A70126
:106BD00096010E94553DDA01C9010196A11DB11D22
:106BE00071C180E00E94192927EE33E0DC010E9488
:106BF0004439A70196010E94553DCA01B9010E947E
:106C00006A2BDFC280E00E941929BC01990F880B12
:106C1000990B0E94093A20E030E040EA50E40E94DB
:106C2000953A2AEA31EF42E85FE30E945F390E9419
:106C3000D139072E000C880B990B0E946A2B80E635
:106C400098E30E94D83083E298E3B9C280E00E94C2
:106C50001929BC01990F880B990B0E94093A20E071
:106C600030E040EA50E40E94953A2AEA31EF42E8E7
:106C70005FE30E945F390E94D139072E000C880B18
:106C8000990B0E946A2B89E998E399C280E00E94DF
:106C9000192990939D0380939C0320919A0330912E
:106CA0009B03AC01421B530B9A0157FF03C0319564
:106CB000219531092139314044F010929503109209
:106CC000940390939B0380939A0360919403709133
:106CD00095036F5F7F4F7093950360939403072E26
:106CE000000C880B990B8BCF80E00E9419299093A0
:106CF0009D0380939C0320919A0330919B03821BF8
:106D0000930B97FF03C0919581959109813991402B
:106D1000B4F18FE399E30E94D83064E670E080E03C
:106D200090E00E9430298FED98E30E94D83064EF04
:106D300071E080E090E00E94302913E00E94473D1E
:106D40002AE130E040E050E00E94553DCB010E9436
:106D5000102B64E670E080E090E00E943029115032
:106D600069F780919C0390919D0390939B0380937E
:106D70009A0364EF71E080E090E00E94302914E013
:106D80000E94473D29E030E040E050E00E94553D40
:106D90000E946A2B64E670E080E090E00E94302957
:106DA000115071F764EF71E080E090E00E943029AB
:106DB00008C280E00E9419298C0190939D03809362
:106DC0009C0380919A0390919B03A801481B590B47
:106DD000CA0157FF03C0919581959109813991406E
:106DE0004CF060E070E0CB010E94B42910939B034B
:106DF00000939A030E94E4299B01AC0180919603C1
:106E000090919703A0919803B0919903281739079F
:106E10004A075B07A1F0CA01B90129833A834B8372
:106E20005C830E94F03229813A814B815C812093FE
:106E3000960330939703409398035093990360917E
:106E40009F0370E080E090E00E946A2B8FE29AE35B
:106E50000E94D8300E94E4299B01AC0180919603E6
:106E600090919703A0919803B0919903281739073F
:106E70004A075B07A1F0CA01B90129833A834B8312
:106E80005C830E94F03229813A814B815C8120939E
:106E9000960330939703409398035093990360911E
:106EA0009E0370E080E090E00E946A2B85EC99E3FD
:106EB00086C10E94473D25E330E040E050E00E945B
:106EC000553DCB010E946B2A7CC180E00E941929AC
:106ED0002CE030E0DC010E944439A70196010E94B9
:106EE000553DDA01C9010196A11DB11D092E000C05
:106EF000AA0BBB0BFC013197ED30F10508F061C125
:106F0000ED52FF4F0C9436398AE296E40E94D83055
:106F100083E096E40E94D8308DE895E40E94D83052
:106F200081E495E40E94D83083E096E40E94D83052
:106F30008FED94E40E94D83083EA94E40E94D83024
:106F400083E096E40E94D83080E694E438C18EE174
:106F500094E40E94D83083EB93E40E94D83084E418
:106F600093E42DC18FED94E40E94D83083E096E441
:106F70000E94D83081EF92E422C180E892E40E941E
:106F8000D83083E096E431C082EE91E40E94D8309C
:106F900086E991E40E94D83083E096E40E94D830DC
:106FA00083EB93E40CC18DE391E426C089E490E483
:106FB0000E94D83081E495E40E94D8308FE090E4BC
:106FC000FEC081EF92E40E94D83088EB9FE30E94DC
:106FD000D8308AE59FE3F3C088E19FE311C089E9D7
:106FE0009EE30E94D83081E49EE30E94D83085E27F
:106FF00092E4E5C080EE9DE30E94D83083E096E401
:107000000E94D8308FED90E4DAC08AE79BE3D7C0C6
:107010008EE19BE30E94D83085E79AE3D0C080E000
:107020000E941929092E000CAA0BBB0BBC01CD0133
:1070300032E0660F771F881F991F3A95D1F722EF2C
:1070400033E040E050E00E94553DDA01C90101966D
:10705000A11DB11D83309105B1F04CF48130910533
:1070600079F0029709F0ADC086ED97E4A8C08430AE
:10707000910561F0059709F0A4C085EC96E49FC0E6
:1070800081E796E49CC08CE797E499C085E297E499
:1070900096C080E00E94192929E030E0DC010E94BE
:1070A0004439A50194010E94553DC901330FAA0B33
:1070B000BB0B8A30910508F084C0FC01E052FF4F01
:1070C0000C9436398AE39BE47AC08DE09BE477C068
:1070D00082ED9AE474C08EE79AE471C084E19AE488
:1070E0006EC080E899E46BC082E099E468C083EBED
:1070F00098E465C08CE798E462C080E398E45FC0E0
:1071000080E00E941929092E000CAA0BBB0BBC01C0
:10711000CD0122E0660F771F881F991F2A95D1F7AE
:1071200022EF33E040E050E00E94553DDA01C90112
:107130000196A11DB11D83309105A1F044F4813069
:10714000910569F00297E9F587E89CE438C084303E
:10715000910559F00597A9F58EEF9BE430C08BECB3
:107160009BE42DC08DE49CE42AC080E29CE427C00F
:1071700080E00E94192927E430E0DC010E944439B4
:10718000A50194010E94553D220F331FF90113C040
:1071900080E00E94192928E130E0DC010E94443996
:1071A000A50194010E94553DF901E15DFE4FE0818A
:1071B000F0E0EE0FFF1FE85BFE4F808191810E949F
:1071C000D8300E946D2702CCE4EBF3E013821282E8
:1071D00088EE93E0A0E0B0E084839583A683B78334
:1071E00080E293E09183808385EC90E095878487AB
:1071F00084EC90E09787868780EC90E0918B808B81
:1072000081EC90E0938B828B82EC90E0958B848B69
:1072100086EC90E0978B868B118E128E138E148ED7
:10722000E1E5F4E01482138215820895991B79E058
:1072300004C0991F961708F0961B881F7A95C9F706
:107240008095089597FB072E16F4009407D077FDDC
:1072500009D00E944B3907FC05D03EF490958195EA
:107260009F4F0895709561957F4F0895EE0FFF1F12
:107270000590F491E02D09940E94A93D332312F466
:107280008A1B9B0B0C9446390E94A93DB7FF0895B9
:10729000821B930B0895AA1BBB1B51E107C0AA1FB9
:1072A000BB1FA617B70710F0A61BB70B881F991FA7
:1072B0005A95A9F780959095BC01CD0108950E943B
:1072C00073390C945B3A0E94543A58F00E944D3A3C
:1072D00040F029F45F3F29F00C94443A51110C948A
:1072E0008F3A0C944A3A0E946C3A68F39923B1F3AE
:1072F000552391F3951B550BBB27AA2762177307DC
:10730000840738F09F5F5F4F220F331F441FAA1F6F
:10731000A9F335D00E2E3AF0E0E832D0915050402B
:10732000E695001CCAF72BD0FE2F29D0660F771FD9
:10733000881FBB1F261737074807AB07B0E809F0BF
:10734000BB0B802DBF01FF2793585F4F3AF09E3F44
:10735000510578F00C94443A0C948F3A5F3FE4F373
:10736000983ED4F3869577956795B795F7959F5F87
:10737000C9F7880F911D9695879597F90895E1E0D3
:10738000660F771F881FBB1F621773078407BA0732
:1073900020F0621B730B840BBA0BEE1F88F7E0958D
:1073A00008950E94D8396894B1110C948F3A0895C9
:1073B0000E94743A88F09F5798F0B92F9927B751D7
:1073C000B0F0E1F0660F771F881F991F1AF0BA9589
:1073D000C9F714C0B13091F00E948E3AB1E008951F
:1073E0000C948E3A672F782F8827B85F39F0B93F11
:1073F000CCF3869577956795B395D9F73EF490953C
:107400008095709561957F4F8F4F9F4F0895E894B9
:1074100009C097FB3EF490958095709561957F4FDC
:107420008F4F9F4F9923A9F0F92F96E9BB2793958A
:10743000F695879577956795B795F111F8CFFAF49A
:10744000BB0F11F460FF1BC06F5F7F4F8F4F9F4FCB
:1074500016C0882311F096E911C0772321F09EE829
:10746000872F762F05C0662371F096E8862F70E08F
:1074700060E02AF09A95660F771F881FDAF7880F69
:107480009695879597F9089597F99F6780E870E03A
:1074900060E008959FEF80EC089500240A9416168A
:1074A000170618060906089500240A9412161306F2
:1074B000140605060895092E0394000C11F4882380
:1074C00052F0BB0F40F4BF2B11F460FF04C06F5F9C
:1074D0007F4F8F4F9F4F089557FD9058440F551F72
:1074E00059F05F3F71F04795880F97FB991F61F046
:1074F0009F3F79F087950895121613061406551FBD
:10750000F2CF4695F1DF08C0161617061806991F28
:10751000F1CF86957105610508940895E894BB271D
:1075200066277727CB0197F908950E94A83A0C9413
:107530005B3A0E944D3A38F00E94543A20F095236D
:1075400011F00C94443A0C944A3A11240C948F3A5A
:107550000E946C3A70F3959FC1F3950F50E0551F50
:10756000629FF001729FBB27F00DB11D639FAA2798
:10757000F00DB11DAA1F649F6627B00DA11D661FE7
:10758000829F2227B00DA11D621F739FB00DA11D08
:10759000621F839FA00D611D221F749F3327A00DC2
:1075A000611D231F849F600D211D822F762F6A2F5E
:1075B00011249F5750409AF0F1F088234AF0EE0FC3
:1075C000FF1FBB1F661F771F881F91505040A9F7F0
:1075D0009E3F510580F00C94443A0C948F3A5F3FE3
:1075E000E4F3983ED4F3869577956795B795F7952C
:1075F000E7959F5FC1F7FE2B880F911D96958795A4
:1076000097F90895FA01EE0FFF1F30962105310515
:10761000A1F16115710561F48038BFE39B0749F161
:1076200068949038810561F08038BFEF9B0741F086
:1076300099234AF5FF3FE1053105210519F1E89449
:107640000894E795D901AA2329F4AB2FBE2FF85F40
:10765000D0F310C0FF5F70F4A695E0F7F73950F053
:1076600019F0FF3A38F49F779F930DD00F9007FCE5
:107670009058089546F00C944A3A60E070E080E833
:107680009FE308954FE79F775F934F933F932F9327
:107690000E94FD3B2F913F914F915F910E94953A3F
:1076A0000C945A3B29F416F00C94443A0C948E3AFC
:1076B0000C944A3A0E94743AA8F39638A0F707F857
:1076C0000F92E8942BE33AEA48EB5FE70E94AB3A6B
:1076D0000F920F920F924DB75EB70F920E94453CEA
:1076E000E4EDF1E00E948C3B4F915F91EF91FF91AF
:1076F000E595EE1FFF1F49F0FE57E0684427EE0FA7
:10770000441FFA95E1F74195550B0E94BF3B0F903E
:1077100007FE0C94B33B0895DF93CF931F930F9311
:10772000FF92EF92DF927B018C01689406C0DA2E03
:10773000EF010E94A83AFE01E894A59125913591A8
:1077400045915591A6F3EF010E94913CFE019701EE
:10775000A801DA9469F7DF90EF90FF900F911F91E5
:10776000CF91DF9108959B01AC0160E070E080E86B
:107770009FE30C945F390C94443A0C94E63C0E94CD
:10778000743AD8F39923C9F3940F511DA3F3915080
:10779000504094F059F0882332F0660F771F881F0D
:1077A00091505040C1F79E3F51052CF7880F911D15
:1077B0009695879597F908955F3FACF0983E9CF0B9
:1077C000BB27869577956795B79508F4B160939533
:1077D000C1F7BB0F58F711F460FFE8CF6F5F7F4F21
:1077E0008F4F9F4FE3CF0C948F3A16F00C94E63CEA
:1077F0000C944A3A68940C94443A0E94743AA8F360
:107800009923C1F3AEF3DF93CF931F930F93FF92AE
:10781000C92FDD2788232AF02197660F771F881F3D
:10782000DAF720E030E040E85FEB9FE3883920F0B2
:10783000803E38F021968F770E947A3CECEFF1E0A1
:1078400004C00E947A3CE9E2F2E00E948C3B8B018A
:10785000BE01EC01FB2E6F5771097595771F880BE0
:10786000990B0E94093A28E132E741E35FE30E9465
:10787000A83AAF2D9801AE01FF900F911F91CF91C3
:10788000DF910E94913C0C945B3AFA01DC01AA0F53
:10789000BB1F9B01AC01BF5728F422273327442785
:1078A000507820C0B75190F4AB2F002446953795FF
:1078B0002795011CA395D2F3002071F0220F331FEE
:1078C000441FB395DAF30ED00C94793C6130710506
:1078D000A0E88A07B94630F49B01AC0166277727F8
:1078E00088279078309621F0208331834283538318
:1078F00008955058BB27AA270E94913C0C945B3AEC
:107900000E944D3A38F00E94543A20F039F49F3FDB
:1079100019F426F40C944A3A0EF4E095E7FB0C9423
:10792000443AE92F0E946C3A58F3BA17620773077A
:107930008407950720F079F4A6F50C948E3A0EF49E
:10794000E0950B2EBA2FA02D0B01B90190010C016F
:10795000CA01A0011124FF27591B99F0593F50F487
:10796000503E68F11A16F040A22F232F342F4427DF
:10797000585FF3CF469537952795A795F0405395D7
:10798000C9F77EF41F16BA0B620B730B840BBAF0A7
:107990009150A1F0FF0FBB1F661F771F881FC2F712
:1079A0000EC0BA0F621F731F841F48F48795779526
:1079B0006795B795F7959E3F08F0B0CF9395880FE0
:1079C00008F09927EE0F9795879508959F3F31F01E
:1079D000915020F4879577956795B795880F911DFD
:1079E0009695879597F9089581E090E0F8940C9426
:1079F000B83D8F929F92AF92BF92CF92DF92EF925B
:107A0000FF92CF93DF93EC01688179818A819B811A
:107A1000611571058105910521F464E279ED8BE52D
:107A200097E02DE133EF41E050E00E94553D4901E0
:107A30005A019B01AC01A7EAB1E40E94743D6B01BD
:107A40007C01ACEEB4EFA50194010E94823DDC0103
:107A5000CB018C0D9D1DAE1DBF1DB7FF03C001974F
:107A6000A109B04888839983AA83BB83BC01CD0157
:107A70009F77DF91CF91FF90EF90DF90CF90BF90F5
:107A8000AF909F908F9008950E94F93C089582E0F6
:107A900091E00E94F93C0895609302017093030104
:107AA00080930401909305010895052E97FB1EF421
:107AB00000940E946C3D57FD07D00E94873D07FC53
:107AC00003D04EF40C946C3D509540953095219523
:107AD0003F4F4F4F5F4F08959095809570956195FA
:107AE0007F4F8F4F9F4F08950E94A93DA59F900DF6
:107AF000B49F900DA49F800D911D11240895B7FF90
:107B00000C94743D0E94743D821B930B0895A1E276
:107B10001A2EAA1BBB1BFD010DC0AA1FBB1FEE1F07
:107B2000FF1FA217B307E407F50720F0A21BB30B52
:107B3000E40BF50B661F771F881F991F1A9469F7CE
:107B400060957095809590959B01AC01BD01CF012A
:107B50000895A29FB001B39FC001A39F700D811D26
:107B60001124911DB29F700D811D1124911D089546
:047B7000F894FFCFB7
:107B7400010001000000002AD432B212251402E1EF
:107B8400C5025F5A050F26FCA5A5D6DDDCFC252B16
:107B940022210FFFF8EEEDEFF7F6FA0003020116CB
:107BA400191A1C1E1F212425272C2E33343536394F
:107BB4003A3B3D3F434445468D2E792E652E512E4A
:107BC4003D2E292E152E012EED2DD92DC52DB12D8D
:107BD4009D2D892D752D612D4D2D392D252D112D81
:107BE400FD2CE92CD42CB42C9A2C842C6E2C4E2CE9
:107BF4002C2C0C2CF62BE02BC02BA52B852B652BCA
:107C04004F2B392B192B032BE32AC32AA32A832AAC
:107C14006D2A4D2A2F2A162AE929BC298F2976296B
:107C24005D292229FA28CD28A02878285F2846280B
:107C34000D28E927BC27A327762749271C27F926DF
:107C4400E026B2268526152E1F1C1F1E1F1E1F1F71
:107C54001E1F1E1FCDDFF10416203B4DC0D4E8FCCF
:107C64001025394DC0D8F0071F374F66B3BFCBD7A7
:107C7400E3EFFB07131F2B37434F5A66C0CBD6E104
:107C8400ECF7030E19242F3A45505B66AEBAC5D102
:107C9400DDE8F4FF0B17222E3945515CAEBCCAD87F
:107CA400E6F4010F1D2B39475563717E929FADBADF
:107CB400C8D5E3F0FE0B192634414F5C00AE80B406
:107CC40080BB40C380CB40D4C0DD80E780F1C0FBE3
:107CD40000064010401A0024402D0036403EC045A6
:107CE400C04C00538058C05D40624066C069C06C9F
:107CF400806FC071C07380750077807EC08280837E
:107D0400C0834084C08440850086808780888089C1
:107D1400C08A008C408D008FC090C092009940A111
:107D240080AB40B840C7C0D8C0EB00004014402727
:107D3400C038C0478054C05E0067406D0010111207
:107D4400131415161718191A1B1C1D1E1F20212287
:107D5400232425262728292A2B2D2F31333536395C
:107D64003B3D3F424547494D4F5155575C5F636624
:107D74006A6E73777B80858A8F959AA000020304CC
:107D840005070A0F142029395172A1FF00000000D1
:0C7D940004278026CD26AB26BF264B27F7
:00000001FF
